:020000041100E9
:103000007FB50023284C294D03932800217C284AB2
:1030100001F0D5FA002812D103232800217C03AA4D
:1030200001F074FA00280AD1224B039A9A4206D181
:10303000214B2248E360224B636104B070BD02263D
:10304000217CFE2228001F4B009601F031FA002857
:1030500001D00020F1E71C4BA2899A42F9D1217CD2
:10306000FF222800194B009601F022FA0028F0D127
:10307000E389174A934203D1164B17486361DCE793
:10308000164A9342E5D1164B164A1B68934206D95D
:10309000C02304222800217C9B0001F072FA124B0D
:1030A00012486361C9E7C046A861FF1FD441FF1FF2
:1030B000813700005959530059598320B4BE00117B
:1030C000F1410011B461FF1F59590000B661FF1FA3
:1030D00083050000A541001194BE00118215000077
:1030E000CC61FF1F87130000AD420011A4BE001188
:1030F000002370B51A4E1B4C30006361637401F0FD
:1031000085F9402323744B2B0CD9CC233821AC22D6
:1031100030009B01217401F034FA00280AD0002508
:1031200025740CE0FFF76CFF051E08D1237C0433E7
:10313000DBB2E7E70C4B0D4D63610D4BE381236878
:10314000002B08D1002D06D00C222900200008F009
:10315000DBFD2B7B6374300001F096F970BDC04637
:10316000D441FF1FA861FF1F4542001184BE00111A
:10317000AAAAFFFFF7B5164B0192C318021D002043
:10318000009388235B05D3181B685C1C1AD09CB283
:10319000402C18D88D781E0CAC466746CD782D0291
:1031A0003D43AE4206D1019800280ED110000C70AC
:1031B000240A4C7003249BB20733A343D218009B0C
:1031C0009A42DED3FEBD4432F9E71000FAE7C0466A
:1031D000FC0F0000802213B503000324019189B283
:1031E000520107319B18A14304305A1A88235B050A
:1031F000C3181B68591C03D190429241104016BD60
:1032000099B2402907D80B000733A343C018904256
:10321000ECD30020F3E74430F9E7134B134A1B6863
:10322000126810B5FA24934201D81A00F824104B02
:10323000E4021B689A4210D813000E4A12689A42A0
:103240000ED3013307D1F823DB029C4203D10A4994
:10325000054808F079FB200010BDFC24E402ECE7EF
:10326000FE24E402F7E7C04600C0071100D00711B2
:1032700000E0071100F00711FFFFFF7FF0B59BB0E2
:10328000150004900391402A00D9A0E006AB5980B4
:103290001A80FFF7C2FF0400042816D9002206A9ED
:1032A000FFF768FF052810D906AB1B88AB420CD18D
:1032B000002D07D0514B2A000499C01808F03CFBA0
:1032C000002802D101201BB0F0BD06AB1D802000FC
:1032D0000699FFF77FFF041E7BD1069B0793FFF73C
:1032E0009CFF80235B01C618802307001B039E42BE
:1032F00001D3F826F60288235B05F31801931B68B7
:10330000013302D0019808F067FB3D49019808F0AD
:103310001BFB3B1D0293331D05938822029B520524
:103320009B181B6808935A1C3CD044219AB2009108
:10333000402A04D80320D11D814389B2009103990A
:103340001B0C8B4224D0402A22D80122300008A92D
:10335000FFF710FF021E1BD1380008A9FFF70AFF74
:103360000400042831D9009A059B9B188022520141
:10337000B218934240D288235B05C118009A09A86D
:1033800008F0C2FC1D4B009A09A9F01808F0BCFA1D
:10339000009A029B9446634402931A4B029AFB18CC
:1033A0009A42BAD388235B05FC1821680198013939
:1033B00008F0CAFA200008F00FFB039A07AB5A8006
:1033C00030000799FFF706FF0400002C03D100200E
:1033D00079E70428FBD988235B05E018069908F0F3
:1033E000B3FA0323EA1C9A4300D16BE7034B049919
:1033F000E01808F089FA65E70424ECE704000011FE
:10340000FFFFFF7FF80F0000F7B505001400402A0A
:1034100021D8002701AE71803780FFF7FEFE042817
:1034200016D93A003100FFF7A5FE042810D93688D6
:10343000BC420BD0BD4209D0221CB44200D9321C80
:10344000064B92B2C118280008F05EFC30B2FEBDF7
:10345000C04300B2FBE703204042F8E7040000113C
:1034600037B5042204000D0001A81649FFF7CCFF70
:10347000020004280BD1019BA34208D3AB4204D025
:10348000104901A80195FFF7F9FE01203EBD0E4C41
:1034900023682000019308F09FFA01992000013968
:1034A000019108F051FA80235B01E418074B9C421C
:1034B000EED10422034901A80195FFF7DFFE0020A9
:1034C000E4E7C0465555000000C007110000081190
:1034D00030B589B008F078FA10226946254808F01E
:1034E000EBF9254B009A9A420ED1019B029A0F2BC1
:1034F00033D8002101240698013B08D2002900D0CE
:103500000292029B013331D10023029325E0551C26
:10351000F2D102002100EFE710341022200004A9AC
:1035200008F0CAF9029B013301D1069B029388235C
:1035300004995B05C918059B06981A03120B0491A0
:103540000592814203D02B4201D108F0DDFB019BA3
:10355000013B0193019B002BDED1029B002B03D08A
:10356000049304984168084709B030BDE025014C38
:103570002D03EFE700000111504859368022F8B5BD
:10358000964C974BD200002120001C6008F05CFB99
:103590002300944A88331A60934B1A786A23002ACE
:1035A00000D01133E3620A232365904B37221B7846
:1035B0000820A3638E4B2118E361102323628D4BF7
:1035C0003B256361C823DB00A36123008C331A60B1
:1035D0002823013AE26320646364CA67043A211D28
:1035E000CA672100BC310D602100C0310860210094
:1035F000C4310B6021000635CC310D602100083D3F
:10360000C8310D602100D0310A602200D432106030
:103610002200D832136022000227E0322100176016
:103620004222DC310A6021001B3DE4310D602100A3
:10363000E83108602100EC310B6023000521F433F0
:1036400019602300F0331A602300183290331A6097
:1036500023009433186023001E3A98331A60AF2376
:10366000DB002360644BFA262363644B644DE36004
:10367000644BF031A3642300FF31FC33B600A1603A
:1036800021611E60A5627325E5656D3D6565A565D3
:1036900096255D4AAD00E264666258606766A5667D
:1036A00000270925A767E566584F594D6067200038
:1036B0002567E2673A6015279C30676007001A208B
:1036C00038602000A0300700212038602000A8309A
:1036D00007004C4838602000F83006602600642758
:1036E000A436376026005F3FAC3637602600033FC4
:1036F000B03637602600C637B4363760260000275C
:10370000B836376038269E60424E96205E64424E40
:103710005A66DE61414E9A645E62F53EFF3E9E62ED
:103720001E269A67354A8000DE661F675F67DD6583
:103730001D661862DA67BE23394A5B00E250394BD6
:10374000D838235004302250C4225200A350C6233C
:10375000E4205B00E1500433334AE1503349344BF9
:10376000D1603449800019503349E938FF38195085
:1037700032490430195032493248D161324911631B
:10378000324951631900F4310860CE2030494000BD
:1037900011603049195019002F48F83108602F493D
:1037A000D16582212E4A89005A501A002D490832CB
:1037B000D1671A002C49B432116088212B4A890044
:1037C0005A501A002A49883211602A4ADA6407F0EE
:1037D000CBFF012008F0C8FAF8BDC0460004FF1F67
:1037E0004464FF1F106FFF1F1844FF1F4A0AFF1F8A
:1037F0003A07000080C3C9019A020000DC050000FE
:103800006A18000050C3000088130000F009FF1F71
:10381000204E00006509FF1F68100000C409000069
:1038200040420F0010270000FC00FF1F751CFF1F07
:103830000000FF1FC92CFF1F5130FF1FE92EFF1F83
:103840003520FF1F2527FF1F5120FF1FFD21FF1FD0
:10385000C11FFF1F4929FF1F312AFF1F8D19FF1F9D
:103860005528FF1F7925FF1F8525FF1FC11EFF1F3C
:10387000791FFF1F391EFF1F0223F0B50124624D7F
:10388000624E2B70624B91B01C70624F0393336891
:1038900000210820FB7006F05BFE082006F052FDB8
:1038A0000023984205D0FA78552A02D0332A00D056
:1038B0009DE03360042006F0C5FF07F0C5FFFFF769
:1038C0005DFE08F031FA1F2201240021524B10AE98
:1038D0001A70524B1C70524B1970524B196891431D
:1038E000163A0A431A60602219689143403A0A4323
:1038F0001A6008F0A1F808F0F7F84B4B9847C12080
:10390000FF214A4B80001A588A431A50C522920060
:1039100098588843BF390143995098584449084002
:103920008021C9010143802099509958C00509029E
:10393000090A0143995080213E48490108F00CF9D9
:10394000032322003C49019400933C4808F074F999
:103950002C223B4905A808F0D7F905AC61782078FE
:10396000023406F00FFDA642F8D1364C00200121AA
:1039700006F01CFE2268344B03201A40A023DB0211
:1039800013432360802322689B041343236022682F
:103990002E4B1A4080239B03134323602C4A2D4B4C
:1039A000934200D8012007F0CFFE08F065F980238C
:1039B0002268DB0413432360287808F0E5F9039BB1
:1039C0001878C0B207F0F8FE07F0FEFE2249042086
:1039D00007F092FF06F002FF00F040F800F024FE2E
:1039E00000F0CCFE00F00CFA002011B0F0BD009306
:1039F0002100194A042008F05FF88023DB059C624F
:103A0000FFF766FD56E7C0464A0AFF1F34F0004044
:103A10001844FF1FD861FF1F480AFF1F490AFF1FF4
:103A2000680AFF1FBCF00040E1A2000000E100E0D6
:103A3000FF00FFFF1C44FF1FA056FF1F1C54FF1F69
:103A4000A8BD001114F00040FF7FF8FFFFFF9FFFAB
:103A50000080FF1F106FFF1F3B000108002210B500
:103A60001100112007F0D0FE10BD0000F8B50023B2
:103A70000926374F374C3B62E3681120B343E360BC
:103A800007F0CAFF112007F08FFF112008F004F99A
:103A90004023226880251343236080236268DB0271
:103AA00013436360A3682C4A2B43A360A3680221DD
:103AB0001340A3608023A2689B0113431022A360DC
:103AC000236C072093432364236C0F3A134323642E
:103AD00080235B003B62226B204B1A402263626BA7
:103AE0001A406263A26B1A40A263E26B1340E36365
:103AF000E3681B4A1340E36006F044FC0121072001
:103B000006F054FD174B11205A6C15435D6407F005
:103B100083FEFD21144B154A89005A508023C7208B
:103B2000626B5B0313436363E36880003343E360CA
:103B30000F4B104A19581140802212020A431A50A2
:103B4000802292051A6008220B4B5A63F8BDC046CA
:103B500000F000403CF00040FFFFDFFFEFFFEFFF11
:103B6000FFFF7FFF003800400000FF1F5118FF1FBC
:103B700000E100E0FF00FFFF0000054070B5284CA9
:103B8000238C002B23D0228A002A21D1DA00238221
:103B90006382A382E38223836383A383E38322601C
:103BA0006260A260E2601F4D1F4A6420EB80934276
:103BB0000AD8FA220020D200934205D91B4A0A21D2
:103BC000981807F0F9FFC0B200232872238470BD53
:103BD0000720E11CCA7F01320240CA7705D10325C4
:103BE000201DC17F01312940C17708325200A35204
:103BF000002321001A00088A01321B180231082A0A
:103C0000F9D1221DD27F9200A350626823689B18CD
:103C1000A2689B18E2689B185B099BB2C3E7C04689
:103C20001861FF1FC061FF1FB70B000030F8FFFFD6
:103C300030B503A804880B20002C0ED14968074D2D
:103C400008784978090201430A20A94205D10121D7
:103C500020001980024B1B7A137030BD192A000016
:103C6000C061FF1FF7B5150008AA16884A680F4FF4
:103C700014785278120222430A24BA4214D1012243
:103C8000DBB2019200962A0007F0F8FC041E0BD16B
:103C9000074B1B68002B07D068782A780002104376
:103CA00042425041013098472000FEBD02290000E9
:103CB0004461FF1F30B5012503790400BFB02B42DA
:103CC00011D00A49408807F045F828420BD0084B2C
:103CD00001A95B8D4D800B80064B00221B7A60880A
:103CE0000B7104F017F93FB030BDC0463C61FF1FB7
:103CF0004840FF1FC061FF1F10B50549054806F089
:103D0000DFFF0421044A054806F09CFF10BDC046B1
:103D10003C61FF1FFFFF0000D4BD00114840FF1FA2
:103D200010B5024804F078FF10BDC046B53C001144
:103D3000012303700B4B1A7A4270022282709A7828
:103D4000C270DA780271032242711A7982715A794B
:103D5000C2710C2202729A794272DB7983720B2053
:103D60007047C046C061FF1F022310B50370013BBE
:103D700043700533837010330371443B43712A331E
:103D800083714433C37100230372064B04001B8804
:103D900043720A30FFF7CCFF831D0A30C0B2E370D4
:103DA00010BDC046C061FF1F10B5142007F024FFEE
:103DB000124B14220021186007F046FF002007F084
:103DC000D3FE012007F0C8FD022007F0A5FF032065
:103DD00004F0C6F9042006F0DBF9052003F004FC2A
:103DE000062004F0D1F8072001F0A8FA082006F018
:103DF00009FF092001F074F810BDC0464861FF1F9B
:103E000007F0BAFD012007F0E7FC07F04DFE0000C7
:103E1000094B10B50400984205D0012904D12000B7
:103E2000064906F04DFF10BD0229FCD1013904F00E
:103E3000B1FE0028F3D0F6E7FEFF00006E61FF1F21
:103E400070B50D7A100004AA2C00168810221440B8
:103E5000154220D1002E20D10A78022A18D14A68B2
:103E6000517815780E4A09022943914205D00D4A2E
:103E7000914209D01C800A2404E014220A491A80C5
:103E800007F042FF200070BD0C2208491A80F7E7B6
:103E90001C800124F6E70824F4E70B24F2E7C0466F
:103EA000F3FF0000F4FF0000A442FF1FD0BE00118A
:103EB00010B504000749084806F002FF074804F05F
:103EC000EBFD0020E40704D50721054A054806F06C
:103ED000B9FE10BD6E61FF1FFFFF0000113E001113
:103EE00018BE00118C40FF1F00B50C4BBFB01A78F4
:103EF0000B4902A800F0FCFC6B4680B2D880002879
:103F000009D06A46074B01A91B889380064B002203
:103F1000188803F0FFFF3FB000BDC0464C61FF1F93
:103F20004D61FF1FE640FF1FF041FF1F00B50C4B26
:103F3000BFB01A780B4902A801F032FF6B4680B27D
:103F4000D880002809D06A46074B01A95B8D938071
:103F5000064B0022188803F0DDFF3FB000BDC046CD
:103F60007661FF1F7761FF1F8C40FF1FF041FF1F2D
:103F7000F7B50E00377A1C0008AB11003D001A8817
:103F800020231D401F423CD13378022B3BD1736864
:103F90001F785B781B023B431E4FBB4208D01E4F6D
:103FA000BB4214D01D4DAB4221D00A252800FEBDD6
:103FB000002A2AD1142C2AD82200F06807F0A4FE87
:103FC000174B1C70012CF1D9FFF7B0FFEEE7002A68
:103FD0001BD1202C1BD82200F06807F095FE114B56
:103FE00004211C70104B187807F056FCDEE7E3B292
:103FF0000124009201940A00310007F03FFB050004
:10400000D4E70825D2E70125D0E70B25CEE70D251B
:10401000CCE7C046F3FF0000F4FF000002290000D7
:104020007661FF1F4C61FF1FF861FF1F332310B53E
:10403000040003700A220749013007F065FE064BB1
:104040000F201B681A0AE37222731A0C1B0E62738C
:10405000A37310BDC061FF1FE861FF1F30B50125CC
:1040600003790400BFB02B4213D00B49408806F0FF
:1040700071FE28420DD06A46084B02A81B88938027
:10408000FFF7D4FF6B46D8800022608801A903F0B7
:1040900041FF3FB030BDC0466E61FF1FE640FF1FCD
:1040A00010B5024804F0B8FD10BDC0465D400011D7
:1040B00070B5160004AA148805AA15784A685078C5
:1040C000117800022A4A0843801805284BD807F0C7
:1040D000DBFB03131E29343F0720042C0BD80522D9
:1040E000121BAA4200D92A0022491A80300009195D
:1040F00007F00AFE002070BD0720112CFBD8122209
:10410000121BAA4200D92A001B491A80EEE7072099
:104110000E2CF0D80F22121BAA4200D92A001749F0
:104120001A80E3E70720032CE5D80422121BAA42D9
:1041300000D92A0012491A80D8E70720032CDAD8C0
:104140000422121BAA4200D92A000E491A80CDE788
:104150000720032CCFD80422121BAA4200D92A0020
:1041600009491A80C2E700220A201A80C3E7C04624
:10417000DCD5FFFF63BE00119461FF1F53BE001129
:104180004EBE001149BE001144BE001110B50D21F4
:10419000024A034806F056FD10BDC04638BE001165
:1041A000FC40FF1F13B5104C0423217C01AA00F032
:1041B000ADF9002815D16B469A88236852BA92B29D
:1041C0005343228909491B0C9B184B806B46DA88A4
:1041D000636852BA92B2534362891B0C9B188B805E
:1041E00016BD0120FCE7C046A861FF1FC061FF1F8C
:1041F00013B5124C06236A46217C00F087F900288B
:1042000019D16B461988236849BA89B24B43218971
:104210000B4A1B0C5B1853806B46D97803335B78D1
:104220001B020B435BBA61689BB24B4361891B0C59
:104230005B18938016BD0120FCE7C046A861FF1FF4
:10424000C061FF1F37B5174C07236A46217C00F079
:104250005DF9002824D16B461B787F2B20D86B4654
:10426000DD78F0232A041B031A406B469B880E4915
:104270005BBA9BB21A4323682D09534322891B0C56
:104280009B184B806B465A789B7812031B011A438C
:1042900063682A43534362891B0C9B188B803EBD85
:1042A0000120FCE7A861FF1FC061FF1F7FB5022648
:1042B000154C0022217C03AB0096050000F0F8F8B5
:1042C000002802D0012004B070BD0E23217C012201
:1042D000280000966B4400F0EBF80028F2D16B4602
:1042E0009A892368D2BA5343228908491B149B1820
:1042F0004B806B46DA89636852BA92B25343628943
:104300001B0C9B188B80DEE7A861FF1FC061FF1F9D
:1043100070B5184C237C002B0FD0382B0ED1164DC6
:10432000280000F073F8CC23AC222800217C9B01EC
:1043300000F027F9280000F0A7F870BDE3890F4AC4
:10434000934209D10C4D280000F060F800222800AB
:10435000217C00F005F9EDE7094A9342EDD1064DC5
:10436000280000F053F890222800217C920100F0F0
:1043700026F9DFE7A861FF1FD441FF1F8305000076
:104380008320000070B5144C237C002B1FD0636980
:10439000002B1CD0114D280000F038F8636928006C
:1043A00098470400280000F06FF8002C10D10C4B47
:1043B0000422995E002905DA9C801A8801321A804D
:1043C000200070BD074A9142F7DD9A80F5E701248D
:1043D000FEF78EFEF4E7C046A861FF1FD441FF1F21
:1043E000C061FF1F0F27000010B58024064AA400FB
:1043F0001168436B234205D113685B1A032BF8D96C
:10440000012010BD0020FCE76008FF1F70B5C179D6
:1044100005000C00631E9C411A4BE402E41849009D
:104420000460C9B2007906F0F7F8E97968794900C3
:104430000131C9B206F0F0F8E8790930C0B207F0EE
:104440002BFC0023E36661332360AA795B3B002ADF
:104450000ED022689A43023B134323600A23E36190
:104460000733236200232363A3630133E36370BD37
:1044700022689A4302231343236046236361063371
:10448000A361EFE70050004070B500250400036809
:10449000DD66C0790930C0B207F0BEFA2900207984
:1044A00006F056F82900607906F052F870BD000059
:1044B000F8B51E0006AB1D78002304681700E366FC
:1044C000616007F081FA01238022E3662B002761F7
:1044D0005200013B08D207F0B7FA08200A4A1168D7
:1044E000002D03D12800F8BD2261F2E7236F0342BB
:1044F00003D02369013D3370013613685B1A032B27
:10450000EED90125EEE7C0466008FF1F70B51C001C
:10451000002305681600EB66696007F055FA012371
:104520008022EB6623005200013B08D207F08CFA90
:1045300008200A4A1168002C03D1200070BD2A61AE
:10454000F2E72B6F034203D02B69013C3370013635
:1045500013685B1A032BEED90124EEE76008FF1FF6
:10456000002370B504681500E366616007F02CFA5B
:104570000123E366256107F067FA2000FFF734FFA7
:1045800070BD70B51D00002304681600E36661600D
:1045900007F01AFA0123E36626610F33626B1A42B1
:1045A000FCD02B0A23611023626B1A42FCD0EDB2BF
:1045B000256107F049FA2000FFF716FF70BD0023C0
:1045C00070B504681500E366616007F0FDF901232A
:1045D000E3662B0A23611023626B1A42FCD0EDB212
:1045E000256107F031FA2000FFF7FEFE70BD70B5BF
:1045F0001E00002305681400EB66696007F0E4F90B
:104600000123A619EB660F33B44205D107F01CFA5B
:104610002800FFF7E9FE70BD21782961696B194216
:10462000FCD00134F0E7000010B5084CE368002B23
:1046300008D18022064B52021B689B186360054B11
:104640001B68236007F040F9A06010BDE861FF1F00
:10465000C8F00040CCF0004070B5184A936A916AE7
:104660009942FBD116498A689A421FD39A1A8B60E5
:10467000144B0126186893B2D202D20E4343424330
:1046800000204C681B0A1B1912029B180E4C0A686A
:104690004B60551CA3420CD8002801D04B600A6027
:1046A0000A4A136008680A4B186070BD581E821AC7
:1046B000DDE7084A30009B182A00EAE700F00040D6
:1046C000E861FF1F140AFF1F40420F00C8F00040BE
:1046D000CCF00040C0BDF0FF70B51F4C23793F2BDC
:1046E00001D93F2323711D4B22791A701878C0B26B
:1046F00007F00AFA18231A491A4A0B801A4913803C
:104700000B805380A379194980200B800C21938062
:1047100001334B43164D191C0001834200D9011C83
:104720002980D1806379002B11D101336371237A01
:10473000012B01D8022323726279237A0D48534357
:104740000A21584307F038FA0B4D286070BDA02BA2
:10475000EDD9A023EAE7C046DC61FF1F480AFF1F2E
:10476000EE41FF1FC443FF1FEC41FF1FEA41FF1F43
:10477000E841FF1F71020000CC61FF1FF8B519214D
:104780000020FEF76DFE114C011E114D09D10C22C7
:10479000104BC1CBC1C4280007F056FAFFF79CFFAD
:1047A000F8BD0C2220000C49FEF72EFE0C2802D08A
:1047B000084B43CB43C40C2228000849FEF724FED3
:1047C0000C28EBD00C220021E5E7C046DC61FF1F7E
:1047D000A861FF1FC4BE0011FC0C0000F50C000016
:1047E000F0B51D4C8022A544040088206946520182
:1047F000400507F0D1F9902212016A44130020000D
:1048000032C832C316C816C38023144C144FA6688E
:104810009B033343A3603B6006F0B6FF8823A06888
:104820005B05C01807F0D8F80025882329008022EE
:10483000A0685B05C01840196944520007F064F88D
:1048400080230135FF355B019D42EED1A6603E60BD
:10485000044B9D44F0BDC046FCEFFFFF3443FF1FF7
:104860009808FF1F04100000F0B5040087B000286E
:1048700025D0684607F030F81B4C022806D10622E6
:104880006946200007F058F8002816D06946002332
:1048900001250F262F00E25C0133100910308740FC
:1048A00038002F00324097403A0002434A610439F1
:1048B000062BEFD16846FFF793FF07B0F0BD182233
:1048C00069460A4807F068F96A46A300D3580133DD
:1048D00005D01822FF21684607F0B6F9EAE701344F
:1048E000062CF1D1E9E7C0466509FF1F0009001158
:1048F000F0B5002504000E0085B0AA4200D186E084
:104900004B1C087801934B78897837790902194351
:10491000F3783F061B040B431F4303972070657019
:10492000252800D196E033D8112813D807F024FAAF
:1049300069002501250125012501AA00B800B10063
:104940002501250125012501250125012501250137
:1049500005011F01232800D1DEE0DB2800D02EE175
:10496000042A00D8ACE01025052A05D0551F2A00DE
:104970003800711D07F0C8F905223100200007F04A
:10498000C3F92A003900601D07F0BEF905353EE085
:10499000562859D010D8332800D19DE0552839D059
:1049A0002628DAD19C4B2900132218001D0007F09D
:1049B0004BF9FEF79DFB5CE0712800D177E072288F
:1049C00000D180E0602800D18BE0DC28C5D1022A2C
:1049D00000D875E07378BFB26370B378A370032A10
:1049E00005D0033A390092B2F01CFEF747FC1022C2
:1049F0003900E01CFEF708FDC51C002807DA6070CE
:104A00005CE00C222000854907F07EF90C25280087
:104A100005B0F0BD013A824D0C2A13D8002A0AD005
:104A20002800019907F070F9FFF756FE0C222800C4
:104A30007C49FEF723FC29000C22601C07F064F976
:104A40000D25E4E70C22EBE7754D774B2A0043CBAD
:104A500043C2E9E7013A704D0C2A11D8002A08D068
:104A60000199280007F050F90C2228006F49FEF741
:104A700005FC29001322601C07F046F91425C6E73F
:104A80000C22EDE706226A49601C07F03DF9062575
:104A9000BDE712226749601C07F036F91325B6E717
:104AA00008226549601C07F02FF90925AFE77178E6
:104AB000F02905D8614B188801F0CEFD0225A6E744
:104AC000FF236370FAE75E4B012A03D072789A7075
:104AD0006270F3E79B78F4E72000FFF7A7FA050080
:104AE00095E7013A564B574D062A10D8002A10D0A8
:104AF000012128005970019907F006F901F062F8C8
:104B000029000622601C07F0FFF807257FE7062230
:104B1000EEE700225A70F3E7042A04D94A4D2F60C9
:104B200006F0D2FEA860FFF797FD0422039003A9C8
:104B3000601C07F0E9F8052569E7444D062ADFD92E
:104B400006222800019906F0F7FE0028D8D0062298
:104B50000199280007F0D8F806223D492800FEF701
:104B60008DFB0123364A91780B439370C8E7012AE5
:104B7000A6D07078FFF778FEA0E7012800D0ECE619
:104B8000931E344F132B06D87378002B0BD100F0F3
:104B900015F900F04BF9304B39001D78601C6A1E86
:104BA00007F0B2F833E7551E2A000199380007F0E4
:104BB000ABF838002949AAB2FEF760FBE9E7DA282A
:104BC0001DD1042A00D87BE7082A15D9B379727958
:104BD0001B021343F27912041A43337A1B06134360
:104BE0003B603B68052231002000039307F08CF8FE
:104BF0000422601D03A956E7FE236370F1E7DE2857
:104C000000D05DE7511E012A01D10025FFE6019881
:104C100000F0BEFFF9E7C046A861FF1FD0BE00113B
:104C2000DC61FF1FFC0C0000C4BE0011F50C00008D
:104C3000B461FF1F9461FF1F3843FF1FF041FF1F46
:104C4000D861FF1F9442FF1FE861FF1F6509FF1F26
:104C5000ADAC0000D963FF1FD763FF1FAEDE0000BD
:104C600070477047020010B5094B0A32094C92B2E6
:104C7000DA815A8298811882207802F053FB04224C
:104C8000054B012120781A7006F006FE10BDC046C3
:104C9000C242FF1F2264FF1F2164FF1F013870B54D
:104CA000042809D806F0F0FD030928081200234B58
:104CB0000221187806F0F0FD70BD204B082118780D
:104CC00006F0E2FF00221E4B1A72F5E78022002454
:104CD0001B4B1A4D52001A8108211A682878DC7281
:104CE00006F092FF2100287806F046FF012000F030
:104CF00087FE00F067FFDFE7104B0821187806F009
:104D0000C3FF1048FFF730F80F4B104A9B79002083
:104D100093800F4A13808022094B5200D8721A8167
:104D200000F06EFE00F04EFF0A4B9B78002BC3D0C4
:104D3000094A136006F0E0FFBEE7C046F861FF1FB6
:104D4000CC61FF1FF941FF1FDC61FF1FC443FF1F40
:104D5000EA41FF1FD861FF1F34F0004010B5012960
:104D60000BD1082809D1054B1B78002B05D0262232
:104D7000034B04485A72FFF775FF10BDFA63FF1F1B
:104D8000CC61FF1FC40900000300F0B50A4D8E1866
:104D9000B14202D152008018F0BD0C782F6824096E
:104DA0003C5D0F271C700C7801313C402F683C5D46
:104DB0005C700233ECE7C046E441FF1F0E22124B49
:104DC00010B51A700D23114C11492370093A043B98
:104DD0001048637006F098FF2D2301220E490F48FA
:104DE000E371FFF7D1FF01220D49FFF7CDFF01224B
:104DF0000C49FFF7C9FF030000200B49020018709F
:104E0000FEF73CFA10BDC046F663FF1FD763FF1FD5
:104E100063BE0011D963FF1F6709FF1FDF63FF1F18
:104E20006609FF1F6509FF1FAEDE000070B5134C59
:104E3000142220001249FEF7E7FA431E114D132BEE
:104E400019D8AB78002B16D0431C2B7009236B703C
:104E500000230019037028780B4B01302900C0B2E1
:104E6000187006F099FF297822000139C9B2002094
:104E700005F006FE70BDFFF7A1FFECE7D963FF1F49
:104E8000AEDE0000D763FF1FF663FF1F10B5114BA6
:104E90001A781870002A0ED000280BD10E4B1A7801
:104EA000062A07D85423D340DB0703D50B4B1878C9
:104EB00002F038FA10BD0028FCD0074B1B78012BFC
:104EC00002D0033B022BF5D8044B0121187806F0E1
:104ED000E3FCEFE7FA63FF1F2164FF1F2264FF1F5B
:104EE00070B5514E514A52493070082005F054FCBB
:104EF0000121022005F05AFB022005F03BFC0121B4
:104F0000002005F053FB002005F034FC00F0E4FE27
:104F1000FEF7EEF806F010FE032246494648FFF77A
:104F200033FF2D24030004221C7044490130FFF795
:104F30002BFF30230470424D424C437083702E3B54
:104F4000062220004049EB87FEF75EFA062813D0C0
:104F5000200006F0C1FC022809D00321200006F041
:104F60001BFD8D23E3706E3B2371193363710622A1
:104F700020003549FEF782F9344B1B68FC335C6432
:104F8000FFF754FF0020FFF781FF314C314A012128
:104F9000314B1278207802F087F9304A304B127882
:104FA0000021207802F080F901222E4B1A702E4B3E
:104FB000DB78552B31D12D4B3B325A722C4B2D4A7D
:104FC000AB81EA812B826A822021307806F08CFE48
:104FD0000120404205F0A0FD0120404205F03CFECA
:104FE000FFF7D4F8FEF788FE00F0B2FC0120404243
:104FF000FEF75EFF012006F08FFCF02001F010FBB1
:105000000121307806F048FC307802F0E7FA1A48BF
:1050100006F062FEFEF72AFD70BD6422174B5B7935
:1050200053431A000A32CBE7F861FF1F614C0011AD
:105030005D4D00113843FF1F9461FF1FB461FF1FD6
:10504000C242FF1F6509FF1FADAC00004464FF1F93
:105050002264FF1F1842FF1FF941FF1FF663FF1F65
:10506000D763FF1FC863FF1FD861FF1FCC61FF1FFD
:10507000C4090000CE090000FA61FF1FDC61FF1FB8
:10508000F8B50A0020230D001A40194263D05E4B88
:105090001B78002B5CD0FFF7DFFA5C4B5C4C5D4E5D
:1050A00099686268737A8A1ADB039A4202D3616054
:1050B000FEF7DCFC327A217A531EDBB2994205D12D
:1050C000FFF726F9002000F0B3FD15E09142F9D377
:1050D00000272772FFF756F9A37ABB4202D0A772C6
:1050E000FEF74CFD012000F0A3FD4B4F3800FEF70A
:1050F0003BFE390006F090FD637A002B25D0013B82
:10510000DBB26372002B20D1444BDB78552B01D1ED
:1051100006F0F2FDE37A002B12D00023A27AE372AC
:105120009A4202D0A372FEF729FD3D4A3A4F1388F6
:10513000380001331380FEF717FE390006F06CFDCE
:10514000642370795843FFF78DFD237A013323726E
:1051500020206840F8BD0BB2002B0ADA314B1878DA
:1051600006F02AFC002801D006F0EEFC80200002A8
:10517000EFE70224214206D0254B01201A72FFF7E7
:1051800085FE2000E5E70B071ED5FFF765FA1F4BEC
:105190001F49204C98684A68637A821ADB039A4256
:1051A00002D34860FEF762FCFFF7ECF8FFF7B0F8B7
:1051B000012000F03DFD00F0E5FB2368DB0701D591
:1051C000FEF76EFF0820C4E7CB0609D5FEF7D6FC34
:1051D0000D4B1B78002B01D1FEF7A2FD1020B8E784
:1051E0000124214207D0104800F06CF806F09CFC26
:1051F00000F004FDC5E70424080020402142A9D0A6
:10520000FEF772FEBDE7C046FA63FF1FE861FF1FAD
:10521000CC61FF1FDC61FF1FF941FF1FD861FF1F39
:10522000C061FF1FF861FF1FDC41FF1FF0B51B4B82
:105230001B4F1B883A8804001A4E1B4D85B09A42BA
:105240000DD832889A420AD3184B1A882B889A4272
:1052500005D1174A174B12881B889A421BD005208C
:1052600001F034FA3B8802AA1380338801905380FE
:105270002B88114D93800F4B02A91B88D3800F4BB5
:105280002A78188802F050FF0D4B08212878019ADF
:105290001C7006F089FC05B0F0BDC046C663FF1F58
:1052A000EE41FF1FEC41FF1FEA41FF1FC463FF1FD8
:1052B000C263FF1FE841FF1F2264FF1FF041FF1F71
:1052C000C063FF1F13B50C4B1C78002C11D10028B4
:1052D00001D00A4B18600A4A0A4B11780A4A107822
:1052E0000A4A01920A4A0092002205F0C1FA2000FF
:1052F00016BD1124FBE7C0462164FF1FBC63FF1FDE
:105300002064FF1F1064FF1F2264FF1FFC63FF1F48
:105310000064FF1F10B5064B12201B78052B06D129
:10532000044B13221988044B187801F0ABFB10BD15
:105330002164FF1FF041FF1F2264FF1F10B50024EE
:105340000122114B52421870104B1C70104B1A80E6
:1053500002F044F904220F4B21001A700E480C325F
:1053600006F07AFB102221000C4806F075FB07229C
:105370000B4B1C600B4B1C700B4B1C700B4B1A70B7
:105380000B4B1C7010BDC0462264FF1F2164FF1F21
:10539000F041FF1F2064FF1F1064FF1F0064FF1F08
:1053A000FC63FF1FD663FF1FD563FF1FF241FF1F82
:1053B000D463FF1FF8B5174C0600257806A81424FF
:1053C0000078052D23D1B41F134FA5B21824BD4278
:1053D0001DD88D1FADB2BD4219D8FA256D00AA4265
:1053E00015D21D000D4F0A3DADB2BD420FD80C4C79
:1053F00026800C4C21800C4900240A800B4A138023
:10540000FFF714FF0A4B0421187806F03DFC20003A
:10541000F8BDC0462164FF1F790C0000750C000028
:10542000EE41FF1FEC41FF1FEA41FF1FE841FF1F54
:105430002264FF1FF0B50BB20D0089B0002B00DB1A
:1054400070E1A44E307806F0B7FA041E50D003780D
:10545000A22B00D122E1D02B1AD0912B45D1437839
:105460000E2B42D19C4B82889A423ED19B4A836844
:105470001278052A39D1032018567F2835D0984B49
:105480001B68002B31D05B68002B2ED098472CE096
:105490008078072829D806F0F7F90428183F3F74C8
:1054A000A8D86378002B0CD101218C4B19708D4B3F
:1054B0001A78002A5BD08C4B307801F0F5FE00287A
:1054C00055D00722854B1A7051E061780029F8D138
:1054D000E378002B11D0854A854B1278307801F0A3
:1054E000E3FE60706378002BEBD1200006F02CFB0C
:1054F00080200002684009B0F0BD784B1B78022B79
:10550000F3D00121307806F077FA0028EAD10121A2
:10551000307806F0C1F9E5E76378002BD1D16F4F01
:10552000032807D13B78052B02D101333B701EE0E5
:105530000223FBE76F4B1A886F4B0293002A0BD0B4
:105540001B78002B03D00121307806F02DFB3B782F
:10555000062B04D1013BE9E7029B1A70F7E7042B05
:1055600041D10121029B3078197006F095F95C4B0E
:105570001B68002BB9D01B68002BB6D0574A107897
:1055800084E76378554F002B27D10622211D5B4805
:1055900006F0BAFB62895A4B5A491A80A2895A4BC3
:1055A0001A80E3890B800521397058490A80584ACE
:1055B0001380228A574B1A80574B1B78012B09D135
:1055C0001F2001F083F8FA22920042430421307830
:1055D00006F0EAFA0022484B75E7312B00D070E75D
:1055E0000022454B1A700323A0E7062200214348FE
:1055F00006F032FA0023454A04211380444A3078E9
:105600001380444A138006F03FFB0821307806F0EF
:105610003BFBA379083B5A425341304A0333137092
:10562000304B1B78002B06D0334B30781A78002A89
:1056300006D001F077FE0122314B52421A8096E7E4
:105640000121197006F028F9F5E70821307806F0F5
:105650001BFB6378002B00D047E72C4B2D4F0293A8
:10566000E388029A04211380294B3078039323891D
:10567000039A138063893B8006F0BEF9002800D0AE
:1056800033E7264B1B68002B00D12EE703990298C5
:105690003A88098800881B68984726E74379132BC6
:1056A00000D022E70389012B0AD11D4B1B78022B66
:1056B00006D10821307806F0E7FAFFF72BFE14E751
:1056C000052001F003F808210200307806F06CFA9A
:1056D0000BE7C0462264FF1F051400002164FF1F72
:1056E000BC63FF1F1842FF1FF941FF1FF663FF1F36
:1056F000D763FF1FF863FF1FFA63FF1FC963FF1F14
:10570000F041FF1FD063FF1FD263FF1FC663FF1F5F
:10571000C463FF1FC263FF1FC863FF1FB863FF1F7F
:10572000C063FF1F8020C001014200D0E2E6CB072A
:1057300031D5324B1B78002B1DD0314E05AC337860
:10574000052B1AD1023B23702E4B21001B782372AC
:105750002D4B1B7863722D4B187801F049FD002802
:1057600009D007202A4B30701B68002B03D01B6820
:10577000002B00D098470120BCE60E20254B0622C6
:105780001B7825492370254B1B78637002ABC0182A
:1057900006F0BAFAD8E7022308001840194209D0E7
:1057A000174B1B78052B03D11D4B188806F01CF8EE
:1057B00002209FE60424214203D0FFF737FD20009A
:1057C00098E6082308001840194200D193E6154BCB
:1057D0001C78012C03D0022C0DD008208AE6124B35
:1057E000124A134913481B881288098800880094BC
:1057F000FFF7E0FDF1E7FFF78DFDEEE7FA63FF1F2E
:105800002164FF1FF241FF1FD463FF1F2264FF1FAB
:10581000BC63FF1FD663FF1FF341FF1FD563FF1F4C
:10582000F041FF1FC063FF1FE841FF1FEA41FF1F58
:10583000EC41FF1FEE41FF1F10B502A804880B20AA
:10584000002C10D1496808784978090201430C48B6
:10585000814209D1022119800A4B59881170DB78E5
:1058600000205BB2537010BD074C0A20A142FAD150
:1058700002211980034B998811705B79F0E7C046CB
:105880006E2A0000C061FF1F6F2A0000F7B51500E7
:1058900008AA16884A680F4F1478527812022243D9
:1058A0000A24BA4214D10122DBB2019200962A00E6
:1058B00005F0E4FE041E0BD1074B1B68002B07D03C
:1058C00068782A78000210434242504101309847DC
:1058D0002000FEBD022900003464FF1F30B5012501
:1058E00003790400BFB02B4225D01449408805F04D
:1058F00031FA28420CD0124B01A95B8D00220B809B
:1059000002234B800F4B5B888B80608802F002FB88
:105910000D49608805F01EFAC0070CD50B4B01A994
:105920001B8800220B8002234B80064B9B888B80B8
:10593000608802F0EFFA3FB030BDC0462C64FF1F14
:105940001C42FF1FC061FF1F2464FF1F7642FF1F20
:1059500010B5074C0749200005F0B2F920000649B0
:1059600005F0AEF90721054A054805F06BF910BDB1
:10597000FFFF00002C64FF1F2464FF1FF0BE001116
:105980001C42FF1F10B5024803F046F910BDC04687
:10599000DD58001170B540253F2608210B4BC2078A
:1059A000D2172A40DD789C7835408C432A439C707E
:1059B000DA70820701D521439970400704D580220F
:1059C000D97852420A43DA7070BDC0469442FF1F34
:1059D00013210A4BDA788A43123901400A43DA70FC
:1059E0000222104202D0D9780A43DA70400703D568
:1059F0001022D9780A43DA707047C0469442FF1FDC
:105A000010B5054B082419790A00A243002801D0DB
:105A100022000A431A7110BD9442FF1F10B5054BB6
:105A20002024D9780A00A243002801D022000A438A
:105A3000DA7010BD9442FF1F0821F8B5324D334B88
:105A4000AE7804000E40AE70984204DD67232B70E0
:105A5000273B6B70F8BD2E4B984203DAE0232B7086
:105A60001A3BF6E700232B706B7083B21A002948AB
:105A70005F3292B2284F82422CD9002C03DA5B426B
:105A80001CB204232B70053420B20A2106F094F8CE
:105A900004B2FA239B009C4232DB08232A7813438A
:105AA0002B706421200006F087F80A2100B206F06E
:105AB000BBF809B22A787B5C13432B700A212000C3
:105AC00006F07AF80A2100B206F0AEF809B27B5C63
:105AD0006A780AE06970002CDBDA5B421CB20423AE
:105AE0002B70F5226B78092CE8DC13436B700A21CC
:105AF000200006F099F809B27B5C1E43AE70A9E75E
:105B0000632CCEDCEDE7C0469442FF1F1B4E000025
:105B10001DFCFFFF2A0800001BBF00110823F7B57A
:105B2000194FCD003E7904001E403E71EDB263284E
:105B300006DD5F3333433B7140231D437D71F7BD69
:105B40000300093305DA20235B4233433B71C6234C
:105B5000F3E70E4B019300280BDA0423444224B2EE
:105B60003B710A21200006F05FF8019B09B25B5CE3
:105B7000E3E70928F5DD0A2106F01EF8019B00B2D3
:105B80001B5C1E433E71ECE79442FF1F1BBF0011DC
:105B9000F8B50A4F05003B780E00002B0CD0084CDE
:105BA0002000FEF733FC33002A0020003978FEF78E
:105BB0001EFD2000FEF768FCF8BDC0463864FF1FDC
:105BC0009C42FF1F70B50A4E0A4D06223100280084
:105BD00005F0B2FE002809D0074C3100062228004B
:105BE00006F092F807212000FFF7D2FF70BDC046F3
:105BF0009442FF1F8E42FF1F8D42FF1FE62220218D
:105C000010B50A4B1A70203A5A701C329A70DA7822
:105C10000A40DA70082219791140033A0A431A71CE
:105C2000B7225A71FFF7CEFF10BDC0469442FF1F46
:105C300010B5244B5B78002B3AD1002838D0224C89
:105C40000223E05E214B1B685B0632D5092332211B
:105C5000584305F0B1FF4130FF3000B2FFF7ECFED2
:105C60000520FFF797FE0422A35E194A63209342A2
:105C700005DC32331800642105F09EFF00B20121DB
:105C8000FFF74CFF237A0024132220009A42604140
:105C9000C0B2FFF7C3FE2000FFF79AFE0D4B187845
:105CA000053843425841C0B2FFF7AAFEFFF78AFF0A
:105CB00010BD0A21053005F07FFF00B2FFF7BCFEE2
:105CC0000320CEE7D861FF1FC061FF1FDC61FF1F0B
:105CD000DD2600002164FF1F70B500250A4C20005E
:105CE000A571FEF793FB11233E212000074AFEF722
:105CF0007EFCA84200D13E35054B20001D700123DB
:105D0000A371FEF7C1FB70BD9C42FF1F0ABF0011CB
:105D10003864FF1F0200F0B501270A480A4E5118E7
:105D20008B1A002B00DCF0BD08241578430868406E
:105D300038404000805B013C58406D08002CF5D194
:105D40000132EDE7FFFF00002CBF0011F0B5002588
:105D50000F269D4200DBF0BD4C5D070944403440F6
:105D6000A400A05801357840F3E70000F0B589B0F1
:105D70006A460D000B000F27110010351C78013307
:105D8000260024093E40167054700232AB42F5D111
:105D90002023024AFFF7DAFF09B0F0BD30BF00113F
:105DA000F0B54E780B7889B036020C0017000190E0
:105DB0001E43012A61D9954B9E4200D877E00133FA
:105DC0009E421CD1062A17D1CA788B7812021A4338
:105DD0000B791B0413434A7912061A438C4B5A6100
:105DE00000221A705A808B4A5A608B4A9A608B4AFA
:105DF000DA60002009B0F0BD88225205EEE7884B3A
:105E00009E423CD182498B78002B00D0F6E00C2AD0
:105E100031D10F22A3789343E278120213432279FF
:105E2000120413436279120613434B60E279A0799E
:105E300012020243207A00041043627A12060243DF
:105E4000CA60E27AA07A1202024376484A8183420B
:105E500008D804236E49142201980B7005F054FFF2
:105E60001420C7E71201D21889235B059A42F0D8A3
:105E700001238B70BDE7022AFAD00523EAE76A4ABC
:105E800001239642E6D1FFF745FA052F0CD9E378B6
:105E9000A2781B021343227912041A4363791B066A
:105EA0001343624A0393136005F026FFA1E7584DA0
:105EB0002B78002B9DD1AB78002B00D1A0E02B8953
:105EC00001339BB20093B34200D091E0132AD4D99E
:105ED000CF7C8B7C3F02122120001F43FFF71AFF6B
:105EE000874200D08EE0002E3DD1E378A2781B02DD
:105EF00013432279E96812041A4363791B0613439A
:105F000003930A228B4212D1FF23A370E370237103
:105F100063716B89002B09D1E37B227C1B02120485
:105F20001343A27B13431B0901336B8100226B894E
:105F3000002B8ED0002A67D1686837013818000B13
:105F40006B6900030390984205D9686105F044FD30
:105F5000EB780133EB7068681022A11C381805F04B
:105F6000D3FC2E8145E76F89009A7B1E9BB293423A
:105F70003AD1E278A37812021A43237905A81B04C8
:105F8000134362796C6812061A43EB68009203921D
:105F9000211D0C22049305F0B7FE0120260004A960
:105FA00040421036FFF7E2FE013F012F17D1009A61
:105FB0000B232861824200D04CE704221C492000B8
:105FC00005F0A2FC042203A9686805F0E5FDE96874
:105FD000039AFF23914200D13CE7F73B3AE73100B7
:105FE000FFF7C4FE1036DFE70923B742A4D831E734
:105FF000009BB34200D9FCE607232BE7022329E7E5
:10600000032327E7062325E70A2323E7FFFE0000F3
:10601000A442FF1F00000111FFFF00005048593645
:1060200001FF0000FFFF001102FF000034F00040FC
:10603000B042FF1F10B5034C0B000122210000F0FD
:106040006BFA10BDF56100110B8870B506000D00EC
:106050000224162B11D92B000322094900F05CFA07
:10606000041E0AD1074B2A881B88191C934200D9A9
:10607000111C300089B200F0EFFA200070BDC0465C
:10608000216200114A64FF1F10B54A780400013AEA
:106090000B000220012A07D80A78002A04D0052222
:1060A0002000024900F038FA10BDC0464F620011CE
:1060B0000A7810B50B0004000220002A04D0072241
:1060C0002000024900F028FA10BDC046FB62001112
:1060D0000A7810B50B0004000220002A04D009221F
:1060E0002000024900F018FA10BDC046616300119B
:1060F00010B5034C0B000B22210000F00DFA10BD6F
:106100009163001110B5034C0B000D22210000F02B
:1061100003FA10BD0364001110B5034C0B000F22ED
:10612000210000F0F9F910BD5D6400110A7810B586
:106130000B0004000220002A04D011222000024992
:1061400000F0EAF910BDC0466D640011002310B5DF
:106150001322190000F0E0F910BD000010B5034C47
:106160000B001722210000F0D7F910BDBF64001109
:10617000002310B51922190000F0CEF910BD00005F
:1061800010B5034C0B001B22210000F0C5F910BD17
:10619000F9640011F7B584890D0006000121002C77
:1061A00022D000238268D3561778002B1EDA0C2CDD
:1061B0001AD90C3CA4B2131940880093230002F0B2
:1061C00086FE431E984101307B06DB0F6B703F2338
:1061D000013C1F40A4B22870AF70AC80002C07D0E7
:1061E000B3680133AB6000210800FEBD0020EBE77F
:1061F000AC60F8E70B7803704B8843704B881B0A40
:1062000083700B79C370042070470420022B06D1E1
:106210000020537811781B02009A0B4313807047BB
:106220000B8803700B881B0A437002207047042000
:10623000009983420AD1537810781B0203430B80E4
:10624000D37890781B02034300204B807047F8B549
:106250000D004B7801240021461C03702B788B42E3
:1062600001D82000F8BD6B78B01C4F1C012B10D159
:10627000890069184B88022233704B88B9001B0AC9
:106280007370691805F068FA04360434A4B2F9B2E0
:10629000E4E7122359436B185A88043132705B8843
:1062A00010221B0A7370691805F056FA1236123460
:1062B000ECE770B5049D14001E00052B01D80420E6
:1062C00070BD637812781B0213432B80E378A278A9
:1062D0001B02134302226B802A71211D681D063E9A
:1062E00005F03AFAB2B22A81E92AE8D82800A11DBD
:1062F0000A3005F031FA0020E2E7002310B50A78F1
:106300009A4201D8900010BD9A008A18548801332F
:1063100004705488DBB2240A447094888470928894
:10632000120AC2700430EAE710B51100029C062B75
:1063300004D004201022142B01D010BD022222719F
:106340004B7808781B0203432380CB7888781B02A4
:10635000034363800431601D05F0FEF90020ECE783
:1063600010B50C788B7804315C43E4B203702200E2
:10637000013005F0F1F9601C10BD0420022B06D19C
:106380000020537811781B02009A0B43138070474A
:1063900010B50C000A88023105F0DEF9208810BD26
:1063A00070B504000D0004981100012B01D80420E1
:1063B00070BD167852781202324302800200F13228
:1063C00055701470E125002C00D10C35023B9AB2B7
:1063D0004280AA42EBD80231043005F0BDF900201A
:1063E000E6E70420009983420AD1537810781B0213
:1063F00003430B80D37890781B02034300204B802B
:10640000704710B50C000A88023105F0A5F9208804
:1064100010BD000070B501211E000420049C0E4038
:106420000B4218D1CB40DDB28D4214D90A49DBB200
:10643000098899420FD32300EE331D7033005800B2
:1064400011184978165C0902314301332152D9B23F
:106450008D42F4D8002070BDBC42FF1F10B50C0067
:106460000A88023105F078F9208810BD10B50C7843
:106470008B7804315C43E4B203702200013005F0F4
:106480006BF9601C10BD10B511000298032B01D8E8
:10649000042010BD14785278043B1202224302807B
:1064A000CA788C781202224342809AB28280EB2A08
:1064B000EED80431063005F04FF90020E9E710B5B9
:1064C0000C000B8803700B881B0A43704B88837089
:1064D0004B881B0AC3708A880430063105F03CF9EA
:1064E000A088043080B210BD0420012B03D100200D
:1064F0001378009A1370704710B50C000B88037066
:106500000B881B0A43704A880230043105F024F9D5
:106510006088023080B210BDF0B589B003931E4B85
:10652000029242000700D05A019102F020F8132590
:10653000061E2DD0029B01240370019B002B04D06A
:10654000001903999847001984B26B461B7A5BB215
:10655000002B0FDA1021380002F01CFB192500284F
:1065600013D130003219E1B202F066FC051E0CD1E5
:106570000C34A4B2042304AA380005A9938006961B
:10658000948101F0AFFD051E02D0300005F024FB20
:10659000280009B0F0BDC0464864FF1F70B5050073
:1065A0000C0000280CD00020814209D010222000CD
:1065B000044905F0D1F801202B7823736B786373BD
:1065C00070BDC04670BF0011F0B506000D00170089
:1065D0001C0085B002291BD00020102907D1022BF6
:1065E00007D0102B03D115E00020102C08D005B0E7
:1065F000F0BD69463800FFF7D1FF2A0069460BE07D
:1066000069463000FFF7CAFF22006946380004E0FF
:10661000022BE9D12A003900300005F025F9E6E720
:10662000031CF02800D9F023032008499AB2013A4C
:106630000B80D317034006499B189B100B80D30F88
:1066400004499B185B100B807047C046C042FF1F77
:10665000BE42FF1FBC42FF1F034B1B888B4202D36D
:10666000024B4000C1527047C042FF1F4864FF1FE9
:10667000014B4000185A70474864FF1F1722014B16
:106680001A8070474864FF1F70B505000E2005F0A2
:10669000ABF9041E13D0D0230370002306228370AD
:1066A00007494570033005F057F8064B2100DA8A98
:1066B00062811B7E2373044B187805F03DFB70BD8F
:1066C0006464FF1F5464FF1F1043FF1F262803D874
:1066D000024B4000C05A70470148FCE7C242FF1F0E
:1066E000FFFF000070B506000C00094D1C220021C0
:1066F000280005F0B1F9074B1E70074B1C7005F020
:1067000023FB0123002801D0002312202B7070BD31
:106710005464FF1F1043FF1F7564FF1F70B5050011
:106720000D4C0800E260A16010220021656005F0B8
:106730007BF8012803D11021A06802F058FD102237
:106740000021280005F070F8012803D110216068AD
:1067500002F04DFD70BDC0465464FF1F70B5041EAD
:1067600005D1002903D006220D4804F0F5FF0D4B9A
:106770001D78012D11D1002C05D102221A7005F0CF
:1067800003FA280070BD00221A70074B1B78FF2BFC
:10679000F7D02000FFF778FFF3E70025F1E7C046C8
:1067A0006464FF1F5464FF1F1043FF1F030010B5F4
:1067B000002801D1002010BD00780B4A002803D129
:1067C0005988D1821B7913761378022BF2D10023DA
:1067D000984200D103331370044B1B78FF2B01D078
:1067E000FFF752FF0120E6E75464FF1F1043FF1F2D
:1067F000002911D000280CD04B79012803D1402268
:106800005242134303E03F221340032802D00120E9
:106810004B7170474022F4E70800FAE770B5094D64
:106820000100287800280BD0074C0622200004F035
:1068300093FF21002878FFF7DBFF200005F02CF9FB
:1068400070BDC0467464FF1F4E64FF1F00290AD04C
:10685000012808D13F224B799343C02B03D0403B02
:106860005A425341981C704770B5174D06002B785B
:10687000FF2B15D00A2005F0B7F8041E10D0D02346
:106880000370C83B8370114B11491B784670C3706D
:106890000622043004F060FF2100287805F04CFA4D
:1068A0000C4B1B78012B0DD10B4B1B68002B03D01D
:1068B0009B68002B00D09847084B04211878084AA1
:1068C00005F0A2F970BDC0461043FF1F7464FF1F9E
:1068D0004E64FF1F7064FF1F9C64FF1FA064FF1FB6
:1068E00060EA0000014B98687047C0465464FF1F7F
:1068F000014BDB68186870475464FF1F074B10B5E5
:10690000DA68136801331360054B1878FF2803D049
:106910008021C90104F0C0FF10BDC0465464FF1FB0
:106920001043FF1FF7B50E0002F0C8F8051E1CD07B
:106930000E4B06621F78002F00D10778AB7910202C
:10694000019305F051F8041E0FD0D0230380C73BFC
:106950008370019BE91DC3700622043004F0FCFE25
:1069600021003800E66005F0E7F9F7BD0E43FF1F90
:10697000014B18787047C0467464FF1F054B002810
:1069800005D1054B1A78054B002A00D1014B1800A0
:106990007047C0466464FF1F7464FF1F4E64FF1F8E
:1069A000014B58687047C0465464FF1F024B18687B
:1069B000431E9841C0B270477864FF1F421E030017
:1069C0000120152A03D9FF3B5A425341D8B27047E0
:1069D000F0B51C0000230E0085B0039002920B70EE
:1069E000029A934201D3002019E0E55C5A1CD2B20E
:1069F000002DF8D0029851198142F4DC0233DFB245
:106A0000A35C18000193FFF7D9FF002807D0013DD0
:106A1000019A0399EBB233708A4202D1E01905B0B2
:106A2000F0BDDB19DBB2DBE710B50C0002F09EF81D
:106A300003001220002B03D02100588804F00CFF23
:106A400010BD000070B50E4D84006359002B15D0A9
:106A5000186A002801D005F03FF82B59586A002821
:106A600001D005F039F82B59986A002801D005F0BB
:106A700033F8285905F030F800232B5170BDC0467B
:106A80008464FF1F1C4B70B504000E001500994272
:106A90000AD11A4B1B68002B01D1122070BD1B6854
:106AA000002BFAD09847F9E7154B994215D1134BB3
:106AB0001B68002B0AD01B68002B07D098470028C2
:106AC00004D1104B1C70104B1D70E7E7290020000B
:106AD000FFF7AAFF0028E1D1F3E7080001F0EEFF7D
:106AE0000028DAD003780320A342D7D12900300050
:106AF00004F0B2FED2E7C046FEFF00008064FF1F34
:106B0000FFFF00007D64FF1F7C64FF1FF7B50400DA
:106B1000808801F0D3FF0025A84203D00578A08823
:106B200002F008F81C4E3378002B1FD0AB421DD169
:106B30001A4B28001978FFF777FF002818D0002398
:106B40003370A3790820A778A688019304F04CFF3E
:106B5000011E0DD0D0230370CA3B8370019B477088
:106B600086808371280005F0E7F801E0002DE8D168
:106B7000A0880B4B8200D358002B01D0FFF762FF97
:106B80001721A088FFF768FDA08801F027FDA088E5
:106B900001F0FEFDF7BDC0467D64FF1F7C64FF1F52
:106BA0008464FF1FF0B587B01D000CAB1B88070085
:106BB00001930DAB1B88142002930EAB1B881600AB
:106BC00003930FAB1B880091049310AB1B880593B4
:106BD00004F00AFF041E1AD0D0230370CB3B477089
:106BE0008370C670062229000430002D11D004F0F5
:106BF000B3FD019B21006381029B0098A381039B4D
:106C0000E381049B2382059BA37405F095F807B0EC
:106C1000F0BD04F021FFECE7F7B5009308AB1B884B
:106C200007000C200D001600019304F0DDFE041E89
:106C300013D0280001F042FF00280FD00078D023A5
:106C40002370C93BA370009B21002381019B6770C7
:106C5000A580E680638105F06FF8F7BD014B1878D9
:106C6000EDE7C0461043FF1F13B504006489038994
:106C7000C2888188C0780094FFF7CEFF13BD000062
:106C800010B5044C2068002803D004F025FF002331
:106C9000236010BD8864FF1FA122F0B58188920097
:106CA0004A43384B384F1B6804009B189D229200C2
:106CB0009B18827989B01A603B68002B5FD01D78E1
:106CC000324B1B68002B04D05B68002B01D00020E6
:106CD0009847260008363100E079FFF7B7FD237D9D
:106CE000E0710200E0780493638A29000393238A09
:106CF0000293E3890193A38800933300FFF752FFC7
:106D0000E378002B0BD1E289A379A1880292019646
:106D1000E27928000092012201F0DAFEE0703B687F
:106D2000002B20D0FFF7ACFF194D287800281AD08F
:106D3000184B1978FFF778FE002814D02B78E678E6
:106D400008200793A78804F04FFE011E09D0D02326
:106D50000370CA3B4670837087808671079804F081
:106D6000EBFF00232B701721A088FFF775FCA0888C
:106D700001F034FCA08801F00BFD09B0F0BD064B1A
:106D80009DE7C0463409FF1F8864FF1F9C64FF1FF6
:106D90007D64FF1F7C64FF1F1043FF1FF8B50700D1
:106DA00008000E0001F08AFE041E18D02620FFF70E
:106DB0008DFC051E00D12578062004F015FE041E6A
:106DC0000DD00021062204F047FED0232370C23BE1
:106DD00021006770A370A680E8B204F0ADFFF8BD93
:106DE000F0B585B001930AAB1B78070002930BAB9B
:106DF0001B7808000D000092039301F05FFE061E51
:106E000022D0102004F0F0FD041E1DD0102200211D
:106E100004F022FE2620FFF759FC002800D130782C
:106E2000D0232370C13BA370009B21002372019BE0
:106E300067706372029BA580A372039BC0B2E3726A
:106E40000C9BE36004F078FF05B0F0BDF7B50D00D2
:106E5000019001F033FE071E20D00E2004F0C4FD87
:106E6000041E1BD02620FFF731FC061E00D13E7801
:106E7000D0232380C53B0622A370F91DE01C04F03B
:106E80006BFC019B2A0063810123DD401A401D40F9
:106E9000210022736573F0B204F04EFFF7BD0000CD
:106EA000F0B585B0029010000D0017000A9E039304
:106EB00001F004FE041E31D0029B002B2ED1039B57
:106EC00002795B0724D5122313430422002E08D134
:106ED0000B99002905D10C99002902D10D9900299F
:106EE0001AD01A430D9B2271002B00D0C9E0002E4E
:106EF00000D1CFE0002D00D0CCE0606A002801D0A6
:106F000004F0EAFD1C21300004F0A6FE606205E0FA
:106F100002239A430E33D7E793432371654BBA009C
:106F2000D458002C00D1AAE0002E10D0236A002BE8
:106F300003D11C2004F060FE20625E4BBA00D358DF
:106F4000186A002803D01C22310004F005FC0C9BB9
:106F5000002B12D0574CBB001D596B6A002B03D17C
:106F6000162004F049FE6862BB00E358586A002806
:106F700003D016220C9904F0EFFB0D9B002B11D0CF
:106F80004C4DBC006659B36A002B03D1142004F0A9
:106F900033FEB0622B59986A002803D014220D9951
:106FA00004F0DAFB380001F089FD051E67D0414B83
:106FB000BA00D358002B62D01A6A3420002A00D1BC
:106FC0001C389A6A002A01D0143080B20B9A002A29
:106FD00001D01C3080B25B6A002B01D0163080B229
:106FE00004F002FD041E4AD01822002104F034FDF2
:106FF0002620FFF76BFB0190002801D12B7801932D
:10700000D0232370029B200063700A23294EA370B3
:10701000039BBD00A371AB59A780196A18300029E2
:1070200005D01C22A06004F097FB20003430735977
:10703000996A002907D0030014221433E0600293F8
:1070400004F08AFB02980B9B002B08D003001C2243
:107050001C330B992061029304F07EFB0298735954
:10706000596A002903D01622606104F075FB6B4653
:107070002100187904F060FE3800FFF7E3FC05B04A
:10708000F0BD10220D9B0D991B69A018236204F01E
:1070900063FB2CE70B9B002B00D13FE7012D00D0B9
:1070A0003CE7606A002801D004F016FD1C210B9813
:1070B0002AE7C0468464FF1F10B5044C20680028EE
:1070C00003D004F009FD0023236010BD7864FF1F86
:1070D0000B4B07B51A68002A01D100200EBD694686
:1070E000531C012012780731FFF772FC0028F4D0FE
:1070F00002780123100018401A42EED0EEE7C04695
:107100009464FF1FF0B51F4F01203B6887B0002B30
:1071100025D09B78059300F0B3FB002821D00A20EE
:10712000FFF7D4FA04000B20FFF7D0FA164B050046
:107130001E78731E9E413B68F6B2191DD878FFF782
:1071400057FB3B682900DA7A043303929A7901935A
:107150000292009033002000059A04F04DFB07B026
:10716000F0BDFFF7B5FF002805D00620FFF7AEFA07
:1071700004000720D8E70820FFF7A8FA0400092038
:10718000D2E7C0467864FF1F7464FF1F70B50A4ED3
:10719000040033780D00FF2B0DD0042004F024FCF4
:1071A000011E08D0D0230370CE3B45708370C4709D
:1071B000307804F0C1FD70BD2043FF1F70B504009E
:1071C00006200D0004F010FC011E0AD0D02303702D
:1071D000CD3B8370054B44701B688580187804F0A4
:1071E000ABFD002C01D0FFF767FF70BD7864FF1F77
:1071F000F8B5264F06003B680D001124002B05D181
:107200000522234B1B78134202D112242000F8BD23
:10721000204A10241268002AF8D01278002AF5D0EB
:10722000DB0719D52B789A1E012A1AD80C2004F0F6
:10723000E3FC132438600028E8D000230A224370BE
:1072400029000670023004F087FAFFF75BFF041E86
:107250000AD0FFF731FFD9E700F012FB0028E1D197
:10726000E4E7002BE2D0D0E70B4B1B78032BCDD10A
:107270001D20FFF72BFA094B18800028C6D0084BB9
:1072800004211878074A04F0BFFCBFE77864FF1FA9
:107290007564FF1F9464FF1F7464FF1F7264FF1FF7
:1072A000A064FF1F60EA0000F7B50193194B1400BA
:1072B0001A78052306000F0012201A4221D0012956
:1072C00020D1154B1D68002D1BD002201F2C18D873
:1072D000002C02D0019B002B13D0104B1F221E70DC
:1072E0006E1C0021300004F0B7FB01992200300031
:1072F00004F032FA310020002C70002F06D004F088
:1073000013FBFEBD064B12201D68DCE704F044FDB4
:10731000F7E7C0467564FF1F9464FF1F2043FF1FFB
:107320009064FF1FF8B50F4E12243368002B17D05E
:107330001B780F3C834213D100250B4F0221387874
:1073400004F0A2FC094B042138781D8004F09CFC59
:10735000074B28001D8033685C7004F055FB040067
:107360002000F8BD7864FF1FA064FF1F8C64FF1F1E
:107370007264FF1F70B5012823D11B4C2388002B9A
:1073800003D01A4A1578002D07D0194B1B68002B23
:1073900002D01878FFF7C6FF70BD3B2B02D93C3BEB
:1073A0002380F9E7134E0221307804F06DFCFA22B5
:1073B0002388920002215A43307804F0F5FB25809F
:1073C000EAE70B4B1B68002BE6D00B4B1B785B07E7
:1073D000E2D5084B0221187804F056FC0022024B3B
:1073E0001A80FFF769FED7E78C64FF1F7064FF1FE8
:1073F0007864FF1FA064FF1F7564FF1FF8B51E4D62
:107400002868002803D004F067FB00232B601B4E84
:107410003068002803D004F05FFB00233360184F6E
:1074200005243B7818002040234221D0154800F065
:107430002BFA3B78234213D0202004F0DDFB286098
:10744000002813D02022002104F006FB202004F0A5
:10745000D3FB041E306005D02022002104F0FCFA8A
:10746000002004E0286804F037FB2C601320F8BDEE
:1074700000F00AFAF4E7C0469464FF1F9064FF1F0F
:107480007564FF1F1443FF1F10B50A4C23681A1EB2
:107490000ED0002808D10130587004F0B5FA002849
:1074A00005D02368002B02D00021FFF787FE0122C0
:1074B000100010BD7864FF1FF7B5274E0500336834
:1074C0000191181E21D05C78244F012C30D1FFF798
:1074D000FFFD002825D02000FFF7F8F80400412820
:1074E00014D91F4B022118781E4A04F08DFB1E4B45
:1074F0003C3C1C80022233685A703B78002B14D12C
:1075000028000199FFF75AFE0120FEBDFA229200E1
:107510004243002AEED0124B0221187804F044FBBB
:10752000E8E7FFF7D3F80200F3E700233B70EBE74F
:107530003B78002BE8D1032004F056FA011E08D056
:10754000D0230370CC3B457083703368187804F007
:10755000F3FBFFF7B1FDD7E77864FF1F7064FF1FEF
:10756000A064FF1F60EA00008C64FF1F10B517497C
:10757000838802008B4220D011D815498B4217D046
:10758000144900205B1899B2012907D89268117834
:107590005A425341D8B2FFF7F9FD012010BD0E4AFF
:1075A00000209B1807229BB29A424041C0B2F5E7E7
:1075B00083681878FFF768FFF0E7836899785A784E
:1075C000090218781143FFF777FFE7E70A20000068
:1075D00006200000F8DFFFFFAFDFFFFF014B187050
:1075E0007047C0462143FF1F10B5064C207001F0C4
:1075F00041FA207804F080FA0521207800F062FD3D
:1076000010BDC046A064FF1F0BB273B50D00002B68
:1076100000DBC4E0884B187804F0CEF9041E0ED0CD
:107620000378912B0FD0A22B00D1A1E0834B1878C7
:10763000FF2852D0210004F07FFB00284DD180208C
:107640000002684076BD43780F2B76D013D8052B07
:1076500070D00E2BEAD18088794B98422BD8794B89
:1076600098421BD8784B9842E0D1A3681878591CEF
:10767000FFF774F838E03E2BD8D18378032B74D011
:107680006CD8012B6ED0022BD0D1704B1B68002B15
:1076900023D05B68002B20D098471EE06C4BC018AD
:1076A0000C28C3D804F0F0F91DC2C2150BC20B0B95
:1076B0000B3223C23C00674BC0180728B6D8664B74
:1076C0001B68002B09D01B68002B06D020009847B0
:1076D0000AE0A3681878FFF7C7F8200004F034FA2E
:1076E000ADE7A068FFF762F800289FD0F5E7A36830
:1076F0001B78002BF1D0554B1B68002BEDD01B687D
:10770000002BEAD0210055489847EDE74F4B1B6806
:10771000002BE2D01B68002BDFD021005048F3E79C
:10772000504B1B68002BD8D05B68002BD5D02100B4
:107730004348E9E7FFF7EAF9CFE780884A4B9842E8
:1077400003D04A4B984200D070E7464B1B68002B91
:10775000C3D05B68002BC0D02100D5E7153B012BBF
:10776000BBD963E7FFF798FAB7E7FFF77DFAB4E70D
:107770003F4B1B78042B07D100236A461380017905
:10778000408800F0C5FCA8E7364B1B68002BA4D04E
:107790005B68002BA1D00100364898479DE7012483
:1077A00021420AD0294B1B68002B04D05B68002BB8
:1077B00001D000209847012043E78B070AD5264BCC
:1077C0001B68002B04D05B68002B01D02000984779
:1077D000022036E70421280008400D4200D131E79D
:1077E000254E3388002B21D0013B9BB23380002BE8
:1077F0001AD1FFF7DBF800280AD0204B1C70164B7B
:107800001B68002B04D05B68002B01D02000984738
:10781000FFF7C6F8694601F001FD6846FEF7FEFF76
:107820001D20FEF753FF308004200AE7024B187832
:1078300004F02AFAF8E7C046A064FF1F2143FF1FA7
:107840000E20000001200000091000009864FF1FB6
:10785000FEDFFFFFAFDFFFFF9C64FF1F0C20000077
:107860000B2000008064FF1F0D200000132000008B
:107870007564FF1FFFFF00007264FF1F7064FF1F2D
:1078800010B501F09BF910BD014B18607047C04660
:107890009C64FF1F0B880020162B01D8172304209F
:1078A000014A13807047C0464A64FF1F002070479A
:1078B000074A03001188814207D09188002099422D
:1078C00002D101308000101870470020FAE7C0464E
:1078D000A864FF1FF0B58F7806000D00C5B01E2FFD
:1078E00015D1FFF7E5FF051E03D10024200045B0A8
:1078F000F0BD00223B003100C078009200F0B2FBE6
:107900000400A81C00F0D2FBFF23EB70EEE7264B2F
:10791000062403931B78FF2BE8D0182FE6D87B08AA
:10792000224A013BDB0002929A589446002ADDD09D
:10793000029AD3185B68002BD8D00878002802D1AF
:107940004B78012B02D10624122FCFD107AFAB8881
:10795000697800976446AA68A047041EC6D1AB7830
:10796000029A5B08013BDB00D318390030005B68EA
:107970009847041E0BD1AB78042BB6D0039A310084
:1079800010782200009700F06DFB0400AEE76A78E3
:10799000002AABD1AA7805A93B88087130000A708B
:1079A0004B80FEF747FBA0E72443FF1F80BF001179
:1079B0001D4B37B5050098420BD000290AD1FFF7BF
:1079C00077FF002805D11948FFF772FF002800D083
:1079D000058037BD01291AD1FFF76AFF041EF8D0D0
:1079E00001235B420380A378FF2BF2D0FE2B07D04C
:1079F0000023E0781422009329001E3300F032FBAC
:107A0000A01C00F053FB01235B426380E1E70229E5
:107A1000DFD1013901F0BEF80028DAD12800FFF7E4
:107A200047FF041EDFD1D4E7FEFF0000FFFF000088
:107A3000022210B5074B52421A80074801325A8081
:107A40009A80DA8000F07EFA044801F025F80020E0
:107A500010BDC046A864FF1FD5780011B179001190
:107A60000388F7B50400002B02D102252800FEBDD3
:107A700042680221137825485268FEF7A5FD0028C8
:107A80002ED0234F01253A88002AEFD08023218869
:107A90005B0201259B1A9942E8DC0C2004F0ACF84B
:107AA000061E31D03B8822889C4600231800019591
:107AB00061469DB2491989B2AA421BD8002801D05B
:107AC00062443A8000233000082208C0210003F0FD
:107AD00043FE104A1368002B13D100251660C5E73A
:107AE0006268022113780C485268FEF76DFD002889
:107AF000C7D1BAE760681D0140194181013301987F
:107B0000D6E71A001B68E6E71325AFE7EEBF0011C2
:107B10002243FF1FA464FF1FECBF0011014B18702C
:107B20007047C0462443FF1F14230A0010B51A40B3
:107B3000194204D00122102101F048F810BD4B0673
:107B4000F9D4012088434000F8E710B514008B06F3
:107B500004D50122102101F039F810BD08230A00D4
:107B60001A40194202D14BB2002B0FDA102101F05A
:107B70002DF8002808D02300F2331B78002BECD01E
:107B8000F1342378012BE8D10020E6E703208907B0
:107B9000FAD4E2E7F0B51F00184B85B01C680190DD
:107BA00002910392002C27D1200005B0F0BDA568FA
:107BB0003301ED186B89019A934211D3029A9342D3
:107BC0000ED8002F04D10A9B002B10D12C00EBE71C
:107BD0003B002978039A6868FEF7F6FC0028F2D18A
:107BE0000136B6B2A388B342E1D82468DAE7A368C5
:107BF0000A9A5B891380E9E70026F3E7A464FF1F74
:107C000037B50C000A8849880123914217D3002A0E
:107C100015D0651D23792A0002210A48FEF7D4FCFD
:107C2000102300280BD023796188208800242A00A3
:107C30000094FFF7AFFF0A23A04200D023001800F2
:107C40003EBDC046EEBF001113B50A000888498842
:107C5000012388420BD8002809D00024137905326B
:107C60000094FFF797FF0A23A04200D023001800DA
:107C700016BD13B50A0008884988012388420BD82D
:107C8000002809D00024137905320094FFF782FF01
:107C90000A23A04200D02300180016BDF0B58BB017
:107CA00003904A8808880E000123824255D3002899
:107CB00053D00023012704AC2370002271881300E5
:107CC0000092FFF767FF051E3ED02078002835D1CF
:107CD0002B78022B18D167706A8983000130E31872
:107CE00080005A8069680222201803F035FD23784D
:107CF0000133DBB22370042B19D93B0068890130B2
:107D000080B2002BD9D01FE00223637012235843A6
:107D10006A89231804305A8069681022201803F0F9
:107D20001BFD23780133DBB22370002BE5D10C4A15
:107D30006B899B185A425341DBB2DFE76378012B12
:107D4000E4D12B78022BC7D022780A23002A04D052
:107D500021000398FEF798F9002318000BB0F0BD3E
:107D60000100FFFF0F4BF0B504001868002816D083
:107D700083685D89A54207D88288AE18B44203DAC9
:107D800012019A18934201D10068EFE71E005F8943
:107D90001036A74204D1002900D00D801800F0BD94
:107DA0003300EFE7A464FF1F70B505000C000888DE
:107DB0000021FFF7D7FF03000120002B04D0220091
:107DC0002800197AFFF7C1FE70BDF7B50C00002539
:107DD00001902300EE331B78AB4201D800200AE06B
:107DE0006B00E65A00213000E718FFF7BBFF0028C0
:107DF00002D126800130FEBD017A0198FFF794FE82
:107E0000002802D03B882380F5E70135EDB2E0E79A
:107E100010B5040008880021FFF7A4FF030001202B
:107E2000002B03D02000197AFFF77EFE10BD000062
:107E3000054B1B68002B01D1180004E09A68528999
:107E40008242F6D198887047A464FF1FF0B50E27D0
:107E5000002687B0039302ABFF183E8005001F4B3E
:107E600040891400984207D02B78013000976A6847
:107E700080B2FFF78FFE060002212B7818486A684F
:107E8000FEF7A2FB00280FD06C892000FFF7D0FF7F
:107E9000002802D0013C0419A4B2039B002B00D09F
:107EA0001C80300007B0F0BD02212B780D486A68B5
:107EB000FEF78AFB0028E7D102212B780A486A687E
:107EC000FEF782FB002807D0002EDED03B88A342BD
:107ED000DBD17489013CDFE76C89DEE7FFFF00003E
:107EE000EEBF0011ECBF0011EABF001110B50C008D
:107EF000FFF7DEFC03000220002B0AD0002C00D08C
:107F000023609B781720FE2B03D00138FF2B00D174
:107F1000002010BD73B50D0001A904001600FFF785
:107F2000E5FF172805D0002E04D129002000FEF718
:107F300027F976BD01221021200000F047FE00281D
:107F4000F3D0F6E7014B18607047C046B464FF1FDA
:107F500037B56B469D1D010004000222280003F086
:107F6000D3FE2B88B02B0ED12379122B09D12300FD
:107F7000FA331B78012B06D10121608800F0E0F86C
:107F800001E01B2BF8D037BD10B5054B042118704C
:107F900000F098F8FFF74CFDFEF770FB10BDC046EF
:107FA000B864FF1F0020F0B50BB20F0087B083420A
:107FB00034DA274B187803F0FFFC051E2BD003782A
:107FC000A02B25D103AE3100FEF7E4F8041E0BD13F
:107FD000B378DB0724D51F4B06341B68002B03D076
:107FE0003100688898470400A868002801D003F091
:107FF000F3FD002C08D1184A039B1340174A934203
:1080000006D0B3781B2B03D00121688800F098F8C4
:10801000280003F099FD80200002784007B0F0BDF1
:108020000F4B1B68002B10D0310068889847041E46
:10803000DAD07378002BD7D1B27801A90A704B80BF
:108040000C716888FDF7F6FFCEE70624F1E7C0461D
:10805000B864FF1FB064FF1F00FFFF0000011200A3
:10806000B464FF1FF7B50190FC200D0017001E003F
:1080700003F0BAFC04001320002C12D0B02320001F
:108080002370089BF4226770658026710830002BEE
:1080900008D0190003F060FB2100019803F04CFEAA
:1080A0000020FEBD089903F0D7FCF5E710B5041ECB
:1080B00006D00078FD2803D803F0B6FCFF23237018
:1080C00010BD00000A1F93B210B504000220032B5C
:1080D00005D882400020024BD1529B189C7010BDE5
:1080E000D864FF1F0B8870B5043B04000D0002200C
:1080F000032B0BD80121200000F04CFD03001420BD
:10810000002B03D02900200000F0DEFB70BD000032
:1081100007B51300034A00920A00012100F02CFC6D
:108120000EBDC0464D83001107B501920322009297
:10813000024B0A00122100F049FC0EBDCB83001156
:1081400007B56B4601AA11800449D8800878063328
:10815000012802D1190003F007FC07BDB964FF1F15
:108160000C4B10B518700023FF210B4A13801381AC
:1081700093819380094A5380137051729381937253
:10818000D174D3821375517703F09EFC00F0FCF993
:1081900010BDC046E864FF1FD864FF1FBA64FF1F0C
:1081A000F0B58DB06B46002003910C229B5E83429C
:1081B00000DBB0E05D4B187803F0FEFB051E00D13C
:1081C000A4E00378902B00D09DE006AF0100468824
:1081D000380000F013FA79680400002900D19CE00F
:1081E0003B88052B6ED13B89032B1CD905AC2000A5
:1081F00000F0A2F86288172A61D83989131D9942C4
:1082000031D17968237804310291D90738D5607863
:1082100000F08EF9071E06D0002303712378012B8E
:1082200008D0132B23D0A868002800D178E003F0F1
:10823000D3FC75E06288029909A800F0A6F80290C4
:10824000380000F08BF909AA2378387A01920022CD
:1082500031000092029A00F012F9380000F064F93F
:10826000029B002BDFD0300000F080F9DBE70378C1
:10827000032BD8D16288029909A800F0D6F8DEE76E
:10828000122B13D1029909A800F0B5F8021EEAD109
:1082900027498B88002BC6D0887909A923780191BA
:1082A00061780091310000F0EAF8BCE7002302AAEF
:1082B00093833000617809AAFFF72AFFB3E71D4BCB
:1082C0000993F6E7042B02D09A1F012AABD8184A6B
:1082D000043B9B00995A0029A5D0D2189078310010
:1082E0003A0000F0AEF800289DD13B88042B03D063
:1082F00001213000FFF724FF012C04D1A8680028D9
:1083000001D003F069FC280003F01EFC8020039BD1
:108310000002434018000DB0F0BD012800D182E7F3
:1083200001213000FFF70CFFEDE7C046E864FF1FB6
:10833000D864FF1F010017000B7803704B7843705F
:10834000CB788A781B021343438070470A88030066
:1083500002700A88120A42700A88012A06D14A88E5
:1083600082704A88120AC27004207047022082423A
:10837000FBD14A8804309A704A88120ADA708A88D7
:108380001A718A88120A5A71EFE710B504000120A9
:1083900082420CD94B780A781B0213432380834214
:1083A00006D1CB788A781B0213436380002010BD6E
:1083B000022BFBD1CB788A781B02134363804B7965
:1083C0000A791B021343A380F0E70B8803700B8824
:1083D0001B0A43704B8883704B881B0AC3708B88C1
:1083E00003718B881B0A4371CB888371CB881B0A6E
:1083F000C3710820704703000120082A14D14A786D
:108400000878120202431A80CA788878120202435E
:108410005A804A790879120202439A80CA79887987
:10842000120202430020DA80704710B504000120D8
:10843000022A05D100204B780A781B0213432380BF
:1084400010BDF8B5060010200F00150003F0CCFA9F
:1084500004000120002C0ED0A0230C222900238030
:108460006780201D002D07D003F076F92100300031
:1084700003F062FC0020F8BD03F0EEFAF6E7F7B572
:108480001E00009008AB142017001D78019103F026
:10849000ABFA041E12D0A2230370019B47704380E5
:1084A000099B057146710C220830002B07D019007A
:1084B00003F052F92100009803F03EFCF7BD099942
:1084C00003F0CAFAF6E737B5041E0FD04388002B35
:1084D0000CD00025C1881323007A1722019500953E
:1084E000FFF7CDFFFF2365806372257037BD000065
:1084F00010B50C4904004A88002A09D08B89002B4A
:1085000005D00020CB8A0222834201D010BD012277
:1085100013000A20434300204032C854C818428048
:108520000472F3E7BA64FF1F0023438003707047AF
:10853000094B00211A0010B55C88002C06D01C796C
:10854000844203D10A234B43D01810BD01310A33B2
:108550000329F1D10020F8E7BA64FF1F10B5040029
:10856000407A03F061FAFF23637210BD7047043054
:1085700010B580B203F080FA002803D004214942EC
:1085800003F012F910BD000070B50025104CA06872
:108590002580A581A580A84202D003F01DFBA5601F
:1085A00000250C4C0C4B606D1D80230058331D7052
:1085B000A84202D003F010FB656500256068002822
:1085C00001D003F009FB013508340A2DF6D170BD46
:1085D0008065FF1F2465FF1F7465FF1F70B5041EB3
:1085E00009D1054D2880A881A880A868002802D05C
:1085F00003F0F2FAAC6070BD8065FF1FF0B54B88E8
:1086000085B00193002343600A7905000F00022A18
:1086100000D07BE0CA88032A17D98B685E78197866
:108620003602DC78D8790E4399781B7A24021B0233
:108630000C43034353495BBA0B80331D93421ED155
:10864000042C04D0631F022B0ED9012015E0019ADF
:108650004D4B1201D35A002B06D00198FFF7BEFFF5
:108660004A4A1369013313610421B8682E812C80B2
:10867000494203F099F86860002005B0F0BD434D11
:10868000042C06D0631F022B0FD9EB680133EB607B
:10869000DBE7019A3C4B1201D35A002B05D001981D
:1086A000FFF79CFF2B6901332B61374B300002939E
:1086B000019B029A1B010193002301998C468B5266
:1086C000130063449C8003939E81FFF750FF039B3C
:1086D000041E986016D00421B868494203F064F87B
:1086E000FA880100043A200003F036F80199029A52
:1086F000FB888A5A043B9B18029A8B522B680133E1
:108700002B60A2E7AB690133AB619EE71E4B02937E
:10871000019B1E01029BF35A002B2DD002998C194C
:10872000A068002828D0012A26D1FA889B189BB27D
:108730007352A189994217D39B1AC018B96803F0E4
:108740000BF8029BA289F35A934200D07DE70022E6
:108750002B81A3882B80A3686B60029BF2520B4A8B
:1087600053680133536070E7084A9368013393609C
:108770000198FFF733FF68E7044A536901335361F7
:10878000F6E7C046EA64FF1F8065FF1FF064FF1F25
:1087900070B5051E15D10B4C0B4B188023005833B8
:1087A0001870606D002802D003F016FA6565250088
:1087B00050356068002801D003F00EFA0834AC424E
:1087C000F7D170BD2465FF1F7465FF1FF0B517005A
:1087D000A12285B0920001934243394B06001B68E9
:1087E0000C009B18D933FF331D78FDF741FF04308F
:1087F000854204DD3000FDF73BFF0430C5B2BD42C9
:1088000007D33A0000213000019B02F0B5FF05B00C
:10881000F0BD2900380003F027FA2300C6B2503318
:108820001E700393019B29006365380003F04CFA26
:10883000CBB20293002B02D0039B01361E700026A0
:108840002300503303931B78B34204D8606D002893
:1088500031D10020DBE7029A2800002A04D0013B36
:108860001000B34200D02800F700E719387003F079
:10887000BBF9786000280ED03A78019902F06CFFBD
:10888000019A3B780136D3180E4A0193D369F6B2A8
:108890000133D361D4E7039B18706065A74205D10B
:1088A000084A1320D36A0133D362B0E7606803F04B
:1088B00093F90834F2E703F08FF900236365C8E702
:1088C0003409FF1FF064FF1FF7B50D0007000421F6
:1088D000686802F069FF2B89040003702B891B0A6A
:1088E00043702B8883702B881B0AC3702E89022546
:1088F0000436F6B2F42E15D81B4B9F4214D10C202F
:1089000003F072F81135011E0CD0902303708E3BDA
:108910000371043B4380154B8460C680187803F0D4
:108920000BFA00252800FEBD5C237B43104AD318B8
:108930000093583301931B78002B0FD103003200B2
:1089400038000099FFF742FF019B05001B78002BC0
:10895000E8D13800009902F06FFFE3E7054A0725E8
:10896000536A01335362DDE7FEFF0000E864FF1F36
:108970002465FF1FF064FF1FF0B587B0009017203B
:108980000F0016000193FFF7F2FD1325041E19D006
:108990000C98031E02D00199201D9847030AE3702A
:1089A000052302AAA0700430908127700098667099
:1089B00003A993800494FFF787FF051E02D02000CF
:1089C00003F00AF9280007B0F0BD0000F0B587B049
:1089D0001F000CAB1B780391059301210DAB060022
:1089E0001C78049200F0D6F81425002821D020002D
:1089F000FFF77EFD0135041E1BD01149059B0A7847
:108A000003700132D2B2131EC68001D101231A00B5
:108A10000B7022713000049B03990097FFF7ACFFA5
:108A2000051E09D1230021000648074A093303F037
:108A300043F9280007B0F0BD002363802370F8E7F6
:108A4000EC64FF1FC784001130750000F8B5050005
:108A50000E00064C064F2368002B02D03100280080
:108A600098470434BC42F6D1F8BDC0469065FF1F5C
:108A7000A465FF1F0123064A5B4253800023137144
:108A80005362044A136053609360D360136170476C
:108A9000A465FF1F9065FF1F0200002310B5064963
:108AA0009C000859002801D1625010BD0133052BEC
:108AB000F6D11320F9E7C0469065FF1F034A53889B
:108AC000181A43425841404210407047A465FF1FA6
:108AD000F0B585B002930AAB1F780CAB1B880090F1
:108AE00008000E0001920393FFF7E8FF0500112034
:108AF000002D1BD10E48FFF7E1FF04001520002CCC
:108B000014D006220B99A771E01D02F025FE019BEF
:108B100030002371029B29006371009B66802370E3
:108B2000039B6562E381FFF791FF280005B0F0BD6C
:108B3000FFFF000010B5FFF7C1FF04000220002C6A
:108B400012D060880121FFF781FF606A002801D000
:108B500002F0C2FF28220021200002F07DFF012345
:108B600000205B426380207110BD000030B5074AD1
:108B7000074C5588010013780020A54204D05B1AE9
:108B800059424B415842104030BDC046A465FF1FBA
:108B9000FFFF0000084A10B501230C00904208D0E6
:108BA000FFF78CFF031E04D0037923405A1E934124
:108BB000DBB2180010BDC046FEFF0000024B187962
:108BC000431E9841C0B27047A465FF1F70B50400F2
:108BD0000D001600FFF772FF002804D10D4B9C42D8
:108BE00000D0143070BD416A03790520002907D0F8
:108BF00012221A40102A02D10520002EF2D10F2095
:108C0000DB06EFD5897E0C20A942894149424942C1
:108C10000840E7E7FEFF0000030010B5002800D180
:108C200010BD0348034A41889142F9D09847F7E7BD
:108C3000A465FF1FFFFF0000002330B5C45CCD5CBE
:108C40006C40D4540133102BF8D130BD0F230022D7
:108C500010B5C45C64002243CA54C25CD209013B13
:108C6000F7D210BD0200010010B52032103102F021
:108C700003FE10BDF0B58BB00390102005931700D4
:108C8000049102F0B9FF0090102002F0B5FF009BA4
:108C900013240190002B05D000280CD11324009838
:108CA00002F01AFF019B002B02D0180002F014FF03
:108CB00020000BB0F0BD102002F09EFF0600102037
:108CC00002F09AFF13240500002E00D1AEE0002828
:108CD00019D01022002102F0BFFE320029000398B3
:108CE00002F0CAFD041E0ED133787F2B51D830001C
:108CF0000099FFF7ABFF009B1B787F2B53D801999E
:108D00000098FFF7A3FF300002F0E6FE002D02D02E
:108D1000280002F0E1FE002CC1D1102002F06CFF0F
:108D20000600102002F068FF0290002E7CD0002880
:108D300078D03A000F3223000125121105D00F33ED
:108D40003B4015B25A4253411BB26A1E1201002B1E
:108D500033D0049BD2B298180099029AFFF76CFFA7
:108D6000013D10220021300002F076FEADB2049FDA
:108D70002D017D19AF4242D0002C33D0300002F0DB
:108D8000ABFE029B002B00D189E7180002F0A4FE85
:108D900085E729003000FFF759FF28002549009A90
:108DA000FFF74AFFA7E729000098FFF74FFF2800C9
:108DB0002049019AFFF740FFA5E70F210F400499D2
:108DC0008A18D9B28F4208D9D15C06A81954013348
:108DD000102BF6D1029A0199C0E7791A4842414115
:108DE000C901F2E73900300006AAFFF725FF32007B
:108DF000039806A902F040FD10370400BAE7002CE2
:108E0000BCD13000029906AAFFF716FF320006A96E
:108E1000039802F031FD082204003100059802F0A9
:108E20009BFCABE71324A9E71324AAE7002800D092
:108E30006EE733E7F4BF0011F0B58BB00F001600FA
:108E40000225009000283FD0002A3DD00B1DDBB248
:108E50001800029302F0D0FE1135041E34D0FDF745
:108E600047FD05003A000099201D02F0ADFEEBB26F
:108E70000393E3702B0CDBB22F0A00936370FFB2F5
:108E80002B0E2370A7700193FDF72CFD102201001B
:108E900006A802F099FE2100029A04AB06A8FFF78B
:108EA000E9FE051E0DD1039B08223370009B04A927
:108EB000B370019B7770F370301D02F085FEFDF7F3
:108EC0001DFD200002F008FE28000BB0F0BDF0B53B
:108ED0008FB00D00149E039004920593002A03D1D5
:108EE000022420000FB0F0BD002EF9D00398FFF748
:108EF000E5FD1424071EF4D07278337812021A4369
:108F0000B3781B041343F27812061A43036A0192E2
:108F1000934201D30133E3D1002D03D03B790124E7
:108F20009B07DED50822002106A802F095FD059BCF
:108F300013240433DBB21800029302F05DFE051E19
:108F4000CFD0059A0499043002F03EFE042231008D
:108F5000280002F039FE3900102210310AA802F070
:108F600033FE2900029A06AB0AA8FFF783FE041E0F
:108F70000FD1082206A908A802F026FE0822311DFA
:108F800008A802F071FC012807D101990398FDF7A8
:108F9000C9FC280002F0A0FDA3E70124F9E70000C6
:108FA00070B51C4C05002368181E10D0002D14D17C
:108FB0001A78002A0CD1981C083202F0CDFB02F07E
:108FC00093FC0135002808D123681D70012070BD75
:108FD0000A331800082202F0BFFB2368002BF5D0EB
:108FE000122002F001FD061E0DD0C123216803707E
:108FF000457002311022023002F0AEFB23683100CE
:10900000587802F099FE206802F066FD0023236084
:10901000DCE7C046CC65FF1FF8B504002020FDF753
:1090200055FB0D4EA700BB590500002B0DD00028A5
:109030000BD0D878FF2809D108492A000C55F359DC
:1090400007480333611802F037FEF8BD290002F02B
:109050009BFC0028F0D1F8E7E865FF1FD065FF1FF3
:1090600071A2001170B5064D84006359002B05D024
:10907000D87802F0D9FCFF226359DA7070BDC0467F
:10908000E865FF1F70B506008CB00C0015000021CC
:109090003022684602F0E0FC31001022684602F0FF
:1090A00093FD1D2021000322684402F08DFD6846D7
:1090B000FFF7D8FD2D21040003222800694402F0A7
:1090C00083FD20000CB070BDF0B50700160097B00E
:1090D00001931CAB1D7830221EAB00910AA8002121
:1090E0001C7802F0B9FC102239000AA802F06CFDCD
:1090F0001022002102A802F0AFFC0722310002A8D2
:1091000002F062FD072202AB9818631E9C41019990
:1091100002F05AFD02AB9C732B005A1E934102AA27
:10912000D3730021102206A802F096FC06221D9996
:1091300007A802F049FD1A2002ABC01806221F99A9
:1091400002F042FD102200990EA802F03DFD10220F
:1091500002AB0EA908781C78013A6040D2B20870C0
:1091600001330131002AF5D10AA8FFF77BFD102257
:1091700012A904000EA802F0EFFA102206AB0EA905
:1091800008781D78013A6840D2B208700133013185
:10919000002AF5D10AA8FFF765FD044310222098A4
:1091A000E4B212A902F010FD200017B0F0BD70B5B6
:1091B0000E0014008CB00100102268461D0002F061
:1091C00003FD3100082204A802F0FEFC2100082261
:1091D00006A802F0F9FC6846FFF744FD04001022DF
:1091E000280008A902F0F0FC20000CB070BDF8B512
:1091F00006000D0000243719AC4200D3F8BD02F080
:1092000053FB030A3B70631CDBB201379D4203D959
:109210000234F054E4B2EEE71C00EDE773B506004B
:109220000C000225002819D0002917D0032101A81D
:10923000FFF7DDFF6B469A793F231A400133134352
:109240006A463000937101A92200FFF71BFF051E3B
:1092500004D10322E01C01A902F07EFA280076BDA9
:1092600003785807DA08C00FD20080009B0710432C
:109270009B0F1843C0B2704707230B40C908C900B1
:109280000B4303707047000070B50400FFF7EAFE5F
:10929000134DA4006359002B21D0186A002801D077
:1092A00002F01AFC2B59986E002801D002F014FC31
:1092B0002B59D86E002801D002F00EFC2B59186FE4
:1092C000002801D002F008FC2B59586F002801D06B
:1092D00002F002FC285902F0FFFB00232B5170BD65
:1092E000E865FF1F0E4B8000C35870B50C00002BC3
:1092F0000FD09D68002D0CD02B78201D0B706B7843
:109300004B70A97CFFF7B8FF2B7E23726B69E3607B
:1093100070BD10220021200002F09EFBF8E7C0463D
:10932000E865FF1F014B18607047C046E465FF1FEA
:10933000074A03008000825810B5002A06D0D08862
:10934000984203D1012901D1FFF79EFF10BDC0460D
:10935000E865FF1FF0B5264E95B087000B93BB590B
:109360000500099112200A92002B31D0D888FFF70E
:10937000A5FB04001420002C2AD0280010A9FFF718
:10938000B1FFBB591E781D6A002E23D00895FDF74A
:10939000EFFA07000020FDF7F1FA0790A379E61D28
:1093A000069310AD0CA9089800F0E2FA0EA9280067
:1093B00000F0D7FA0B9B0A990493069B0998029335
:1093C000079B0396019300970EAB0CAAFFF77CFE58
:1093D00015B0F0BDFDF7CCFA06903000FDF7CEFADF
:1093E000E31DA779079310AB06000893DAE7C046A0
:1093F000E865FF1F30B50C4C85002A59030085B085
:109400000120002A0ED018006946FFF76BFF2B5988
:109410001A78D888054B002A00D1054B6A460721E7
:1094200000F0D9FB05B030BDE865FF1F639900115E
:109430007199001130B5094C8500295985B0102269
:109440006846253102F088F92A591121044BD08849
:109450006A4600F0C0FB05B030BDC046E865FF1F9E
:109460000D9A001130B5094C8500295985B010229C
:109470006846353102F070F92A591121044BD08821
:109480006A4600F0A8FB05B030BDC046E865FF1F86
:109490004B9A0011F7B54D4F86001020F4590D007E
:1094A00002F0AAFBF3592062186A132200286CD03C
:1094B000033A29009C6802F04FF9F3591A78019297
:1094C000002A58D11E6A227D317B944651400122E8
:1094D000019F114201D167461740217D91433943D5
:1094E0002175377B4F40BC4660460027800701D47A
:1094F0004F081740012102208F40227D82433A43CA
:109500002275377B5740BC4660460027400701D490
:1095100097080F400420227DBF0082433A43227502
:10952000627D002794466046727B42400A4201D128
:1095300067460F400121627D8A433A436275777B1B
:109540005740BC4660460027800701D457080F40AB
:109550000220627D7F00824317436775767B00227D
:109560007E40760701D4BA080A400426617D920045
:10957000B1430A4362756A78002A08D06278002AEB
:1095800005D005220533DA7700221000FEBD042243
:109590002979114205D1A17C114202D10533033A48
:1095A000F1E7019A21782C78002A02D10A002100E3
:1095B000140018220429E8D8042CE6D805206043BA
:1095C000034A05331218525CDDE7C046E865FF1F09
:1095D00004C0001110B50A001121024B00F0FBFA83
:1095E00010BDC046A79A00110B0030B587B001AD81
:1095F0002B806B4604001100981D082202F0ACF885
:109600002A000B212000024B00F0E5FA07B030BD24
:10961000CF9A001110B50A001121024B00F0DBFABD
:1096200010BDC046239B001113B50B0011006A4604
:1096300013706B4604000622581C02F08DF86A462F
:1096400008212000014B00F0C6FA13BD439B001116
:1096500010B50A001121024B00F0BDFA10BDC04642
:10966000939B00117FB505000B4BAA00D45808004E
:10967000002C0FD0666F237FE28821780396266F37
:109680000296E66E0196A46E0094FDF709FC280090
:10969000FFF7FAFD7FBDC046E865FF1F10B5172133
:1096A000FFF7E0FF10BD000070B50A000D00064B8B
:1096B0000221040000F08FFA060029782000FFF74D
:1096C000D1FF300070BDC046739A001170B586B0EE
:1096D00000236A461370836804001D78681E0A28F8
:1096E00059D801A902F0D0F8060633373B3F43476B
:1096F0004B4F5300180000F042F9062312284BD0BC
:1097000000281BD16088FFF7D9F90823002813D05F
:109710004279002A47D1264B1A78072312070BD526
:10972000244B1A680723002A06D01668002E03D09F
:10973000290001AAB04703006A4613706B461B78E4
:109740006088002B2AD1FFF767FC06B070BD1800B7
:1097500000F06CF9D4E7180000F087F9D0E71800A2
:1097600000F093F9CCE7180000F0ADF9C8E7180055
:1097700000F0C3F9C4E7180000F0F6F9C0E71800DC
:1097800000F0F6F9BCE7180000F013FAB8E718008B
:1097900000F013FAB4E707236A461370694660883D
:1097A000FFF782FFD1E70523012AC5D1024BB8E7B5
:1097B0007564FF1FE065FF1FE465FF1FF8B52C4FC0
:1097C0008600F35904000D00002B40D0DA88824255
:1097D0003DD15A78062A33D11A78002A2ED001209A
:1097E00099681A6A097D014206D0157B054203D0AB
:1097F00007225A700120F8BD0220014204D0157BD7
:10980000054201D00922F4E70420014204D0127B72
:10981000024201D00B22ECE7164B1B68002BE9D06B
:109820005B68002BE6D020009847BB5900215B788D
:10983000122BDFD12000FFF715FFDBE70E4BECE723
:10984000112A04D1002900D032252900F2E7002D89
:1098500008D12000FFF732F9002803D01023027945
:109860001343037121002800FDF798FAC2E7C046B0
:10987000E865FF1FE065FF1FE465FF1F70B50E4E32
:109880008500AB590400002B13D01B78002B11D19D
:109890000A4B1B68002B04D05B68002B01D0200012
:1098A000984773595B78122B03D100212000FFF7F2
:1098B000D9FE70BD024BECE7E865FF1FE465FF1FB2
:1098C000E065FF1F094B8000C3581020002B0CD00F
:1098D0001A6A002A09D09B68002B06D0127A1B7ED8
:1098E000101C9A4200D9181CC0B27047E865FF1FCF
:1098F00070B503000D0014000220002A30D00029AA
:109900002ED013700B78081D53704B789370FFF7AF
:10991000A7FCE070012002212B7A23716B7B0340AE
:1099200063716A7B0A401343042263716E7B1640A5
:10993000334363716E7BF608F600334363712B7B10
:109940000340A371287B014000200B43A371297BB6
:109950000A401343A3712A7BD208D2001343A37198
:1099600070BD10B50A0001000120FFF7C1FF10BD56
:1099700010B50A0001000220FFF7BAFF10BD70B554
:1099800006000C000220002E30D000292ED0737863
:10999000201D0B70B3784B70F178FFF76DFC01223E
:1099A0003579257271794B100800134093401040AF
:1099B0000343881010408000C9080343C9000B43CB
:1099C0006373B1794B100800134093401040034378
:1099D000881002409200C9081343C9000B4321209C
:1099E0002373FCF773FE854201D2122070BD222042
:1099F000257AFCF76BFE8542F7D823781820042BD4
:109A0000F4D86378012BF1D80020EFE7030010B5FC
:109A10000220002909D0002B07D00322481C0A701D
:109A200019000D3201F098FE002010BD0300022243
:109A3000080010B5002B06D0002904D00E32591CA6
:109A400001F08AFE0022100010BD030010B50220B4
:109A5000002909D0002B07D00422481C0A701900E5
:109A60000C3201F079FE002010BD10B5FFF7DEFFCB
:109A700010BD03000220002906D0002B04D00522CF
:109A800000200A701B784B70704703000220002BE7
:109A900008D0002906D05B7800200B70013B082B12
:109AA00000D918307047030010B50220002909D0F2
:109AB000002B07D00622481C0A7019000A3201F058
:109AC0004BFE002010BD10B5FFF7B0FF10BD020027
:109AD0000B00022010B500290ED0002A0CD007215F
:109AE0001970118859701188090A99701118082283
:109AF000D81C01F031FE002010BD03000A00022036
:109B000010B5002B0CD000290AD09978587809029A
:109B100001431180901CD91C082201F01DFE002079
:109B200010BD030010B50220002909D0002B07D07A
:109B30000822481C0A701900921801F00DFE00203E
:109B400010BD02000B00022010B500290BD0002A26
:109B500009D009211970117818185970511C062262
:109B600001F0FAFD002010BD10B5FFF75FFF10BD3A
:109B700002000B00022010B5002A09D0002907D0EE
:109B80005178197011180622581C01F0E5FD0020CB
:109B900010BD030010B50220002909D0002B07D00A
:109BA0000A22481C0A701900063201F0D5FD002077
:109BB00010BD10B5FFF73AFF10BD02000B000220E8
:109BC00010B5002A06D0002904D018005178FFF7FC
:109BD00053FB002010BDF0B585B017001E006A468B
:109BE00006230500080091819380FEF7C0FC132432
:109BF000011E02900CD03800B047041E05D1280089
:109C000001A9FEF76FFA041E02D0029801F0E4FFEA
:109C10002800FFF701FA200005B0F0BDF0B5040000
:109C20008BB0019115000021102202A801F014FF51
:109C3000334EA700B85900283CD0C388A34239D17D
:109C40000378002B36D14278062A18D10200010091
:109C5000553235310C3006ABFFF7A9FA002829D16F
:109C60002000FFF72FFE020006A902A801F074FDF4
:109C7000200002A902F070F801200BB0F0BD816E47
:109C8000002917D00B8A112A28D19D420ED10198A4
:109C90001231093A01F0E8FD012807D1BB59200033
:109CA0009D6EFFF70FFE29000200DEE73221200043
:109CB000FFF7D8FC2000FEF701FF061E1BD0416A0B
:109CC000002918D00B8AAB4215D108220198123115
:109CD00001F0CAFD01280ED1716A0AE09D42E9D166
:109CE00008220198123101F0BFFD0128E2D1BB59D1
:109CF000996E8A7EB9E7200001F0B6FEBCE7C04647
:109D0000E865FF1FF0B56B4D87007E5985B033784D
:109D100002900393002B00D087E0B368346A01936C
:109D20007078062817D101221B7D134202D0217BB7
:109D3000114218D10222134202D0217B114251D18B
:109D40000422134203D0237B134200D08BE0019BFB
:109D50005A7DEB5991E007380428F8D801F094FDBA
:109D6000032E42678300B36E002B03D11C2001F049
:109D700043FFB066EB599C6E002C1CD010220021D2
:109D8000200001F069FE0298FFF79CFD0100200011
:109D9000FFF72DFA01F088FD208220000821123003
:109DA000FFF725FA0298FFF78DFDA076EB59210009
:109DB000D888FFF70FFC0822EB591CE0B36E002B8C
:109DC00005D01A00198AF0881232FFF70DFC022222
:109DD000019B197DEB5911423DD0207B10423AD0B6
:109DE000073208E0F488FCF7DBFD01002000FFF7F4
:109DF00011FC0A22EB595A70029B9C002A59537895
:109E0000073B042B11D8D088FEF758FE00284ED00F
:109E1000C3895A08D2182849029B0298CB542B595F
:109E200041180433254801F047FF05B0F0BDFCF7A9
:109E30009FFD03000120834201D100200393EB59D1
:109E4000DE88FCF79BFD039902003000FFF7ECFB76
:109E5000019AEB59117D042211420CD0217B114251
:109E600009D00B22C7E7F688FCF73CFD0100300063
:109E7000FFF7EEFB6BE7019A527D01210A4204D005
:109E8000607B084201D00C22B5E702210A4204D0CF
:109E9000607B084201D00E22ADE704210A4204D0C3
:109EA000627B0A4201D01022A5E71222A3E7FA2220
:109EB0005200B0E7E865FF1FEC65FF1F7BA20011B1
:109EC00010B5064B1A780423100018401A4200D02F
:109ED0000348FFF727FA002010BDC0467564FF1F36
:109EE0002843FF1F70B50400FFF7D4FA051E43D1C5
:109EF0002000FFF77FFA234EA400A0598268937CCC
:109F0000DB0708D50321036A1B790B40012B02D123
:109F1000017F0B430377431DD97F8B1E022B0DD886
:109F2000022900D00121C088FCF790FF0421335999
:109F30001A7F59700A431A77280070BD01290CD185
:109F400002231022437000210C3001F085FD3059AE
:109F500010213530FFF74BF9EEE70529ECD102234C
:109F6000D118437010220C3001F0F6FB0423325953
:109F7000117F0B431377EAE708251828DCD1053D4C
:109F8000DAE7C046E865FF1FF0B58BB0059143885E
:109F90007E4F9E00F45915000493002C15D1012921
:109FA00002D000200BB0F0BD101D57781678FFF7D7
:109FB00057F9EB68320002932B7A049901930090D1
:109FC0003B002000FCF70CFFEBE7E388049A934288
:109FD00001D00820E6E72378012B00D1D4E0059BCF
:109FE000581E092800D9CFE001F04EFC05CE0A2901
:109FF000CC506C859AB229000498FFF773FFD1E723
:10A00000200029001022453001F0A6FBB9594B78F9
:10A01000042B02D1013B4B70C3E70B000A00253330
:10A0200035320C310498FFF795F90498FFF702FADE
:10A030000522431E9841BB59C0005A70B2E7200068
:10A0400029001022553001F087FB049B4F4C9D00E6
:10A05000295904980A0006AB55320C31FFF77AF9FA
:10A0600029591022453106A801F0FEFB012808D12C
:10A070000498FFF7F7F90590002804D106222B5920
:10A080005A7005988EE708230593FAE763780C2B3E
:10A090007AD1E36E002B03D11C2001F0ADFDE06608
:10A0A000BB59D86E00286FD01022290001F054FB54
:10A0B000BB590498DC6EFFF705FC0D22A076BB5956
:10A0C0005A706EE7E06E00285ED063780D2B5BD18E
:10A0D0002B8808220382A91C123001F03DFBBB59DA
:10A0E0009A68517D0222114226D0186A407B1042A4
:10A0F00022D00C32E4E763780E2B45D1236F002B7E
:10A1000003D1162001F078FD2067BB59186F002895
:10A1100003D01022290001F01FFB0F22BB59CFE70B
:10A1200063780F2B30D1206F0622691C103001F0AC
:10A1300013FBBB599A68517D0422114203D0196A5E
:10A14000497B1142D5D100210498FFF78BFA28E70B
:10A15000636F002B0DD0BB59586F0028F3D010222D
:10A16000290001F0F9FA0122BB5952425B6F1A61D2
:10A17000E9E7142001F040FDBB5960675B6F002BDD
:10A18000E9D126E72978DFE707200BE7E865FF1F1D
:10A1900010B5064C207001F0FFFA06212078FDF77B
:10A1A00091FF0348FEF778FC10BDC046FB65FF1F1A
:10A1B0003193001100200BB270B50D00834216DA06
:10A1C000264B187801F0F8FB041E0DD00378922B73
:10A1D0000ED0A02B37D0224B1878FF283AD0210080
:10A1E00001F0AAFD002835D180200002684070BD32
:10A1F00043780E2B0BD03E2BEDD18378052B12D05C
:10A20000082BE8D181798088FFF7D8FA08E0154B50
:10A2100082889A42DFD183681878591CFEF7C0FE05
:10A22000002817D1D7E7104B1B785B0712D50F4BCF
:10A230001B68002B0ED09B68002B0BD0C289811DA0
:10A2400080889847ECE7FFF741FAA068002801D022
:10A2500001F0C2FC200001F077FCC5E7FB65FF1FA1
:10A260002143FF1F182000007564FF1FE465FF1FD6
:10A2700010B50078FFF712FA10BD10B50078FFF79F
:10A28000FDFA10BD0C234343084A10B59B185A68C9
:10A29000002A03D0012901D1904710BD9B68002BF3
:10A2A000FBD00029F9D19847F7E7C0461866FF1F91
:10A2B00001238340094A10B5946B1C439463506B8F
:10A2C00098435063D46B20009843012901D12000AA
:10A2D0001843D063116B0B43136310BD0080004023
:10A2E000F0B500240127154B85B0DA6B144E0392AC
:10A2F0001A6C0192DA64019BE3403B4217D0039D44
:10A30000E5403D400295E5B202992800FFF7BAFF0B
:10A31000316A736A002908D03900002B01D00299F4
:10A3200079402800FFF7C4FF01E0002BF9D1013488
:10A330000C36172CDFD105B0F0BDC04600800040C0
:10A34000FC65FF1F064B01215A68C2400A4204D037
:10A350001B68C3401800084070471B6DF9E7C046F2
:10A36000008000400122064B8240002903D0D968BA
:10A370000A43DA607047D9689143D960FAE7C0466A
:10A380000038004030B5032444430F4BE25C1B19F6
:10A390009C785D7801232D1B0135AB40013BA34028
:10A3A000A140DB430C00122807D80849920052183C
:10A3B000116819402143116030BD054A11680B40F6
:10A3C00023431360F8E7C0464BC0001108F000407B
:10A3D00014F00040C21F70B5D4B20623092C0BD86C
:10A3E0000125084C9540002908D00021FFF7CAFF3D
:10A3F00023682B4323600023180070BD2368AB4300
:10A40000F8E7C04600380040214BF0B51B185B78D8
:10A41000022B21D1032444431E4A1F4EA35C121970
:10A420009478012215008540B76B013CE4B23D43AE
:10A43000A240B563194C122815D89B0000290CD1F5
:10A4400017495B1899680A439A600123205C154AF2
:10A45000834011680B431360F0BD11495B18996884
:10A4600091439960F1E70E4B00290DD159690A43D8
:10A470005A61225C1328E8D00123203A93400A490C
:10A48000086803430B60E7E7596991435961F0E7B6
:10A49000FC65FF1F4BC000110080004090C0001100
:10A4A00000F00040A0F00040A4F00040F8B5002407
:10A4B0001B4E1C4D1C4B1B5D012B1FD1194A926971
:10A4C000E2401A420BD00122B25693402200143AC5
:10A4D000D2B2022A09D815494A6913434B610134A3
:10A4E00002360C35172CE5D1F8BD0022B2560F49C3
:10A4F0009200521891680B439360F0E7022BEED163
:10A50000E7B23800FFF71EFF01235840C1B2380000
:10A51000FFF77AFF3800FFF715FF6877DFE7C046DF
:10A520001DC00011FC65FF1FFD65FF1F00F000400E
:10A53000012202388240054B002903D059690A43A1
:10A540005A617047596991435961FAE700380040F0
:10A55000F8B50E0001210F008740114A0400D368AE
:10A56000FD43BB43D360831E8B4201D8FFF7E0FF5E
:10A5700000212000FFF72EFF0A4A0B4B5168012EE5
:10A5800005D139431B1951605E700020F8BD294088
:10A59000516002221C1962709A6915409D61F4E7AE
:10A5A0000038004000800040FC65FF1F012210B50C
:10A5B0008240074B002906D019680A431A6001211E
:10A5C000FFF7C6FF10BD196891431960F7E7C04651
:10A5D000008000400C2370B5002543430A4A29003F
:10A5E0009B181D70094B04001B185D70FFF7B0FF2E
:10A5F0000123A340064928000A681A430A60054956
:10A600000A689A430A6070BD1866FF1FFC65FF1F49
:10A61000348000403080004070B504000E00FF28F8
:10A6200013D003250540FFF7D5FF084AA3089B0078
:10A630009B183F22ED00AA40AE40196820009143CC
:10A64000314319600121FFF78DFE70BD18380040BD
:10A65000F8B50C244443134B0500E4186368002B41
:10A6600003D1A3681220002B1AD0022201270E4B1F
:10A6700000215B195A7028002770FFF769FF636893
:10A680001E1E08D0A3683E00002B04D02800FFF750
:10A6900059FE4640F6B228003100FFF709FE0020BF
:10A6A000F8BDC0461866FF1FFC65FF1FF7B5C42044
:10A6B000FF222B4B80001958002491433F3A0A4354
:10A6C0001A508022274F5202274E1A60274B1D5DD9
:10A6D000002D21D0A31E012B03D80121E0B2FFF7EA
:10A6E00027FF012D18D11F4B9B69E3402B4213D04C
:10A6F000E3B218000193FFF725FE01000198FFF770
:10A7000055FFE3B2143B022B1DD801217156184AA4
:10A710008D405369AB4353613B7F002B0DD0E5B2B5
:10A720002800FFF795FF2800FFF70CFE7B7F010054
:10A73000834202D02800FFF7A5FD01340C37023612
:10A74000172CC3D1F7BD012100237156F3568D405C
:10A75000074A9B009B189A68AA439A60DCE7C046A8
:10A7600000E100E0FC65FF1F1DC00011FD65FF1F3B
:10A7700000F0004010B501210400FFF7E9FE0123BD
:10A78000044A002011194B70A34091690B43936157
:10A7900010BDC046FC65FF1F70B50E00150004001B
:10A7A000FFF718FF0C236343094A20009B189D60A4
:10A7B0005E60FFF74DFFF021064B074A8900051E3A
:10A7C0005A5002D02000FFF705FF280070BDC04698
:10A7D0001866FF1F0000FF1FE1A2001170B5134DA6
:10A7E00007202C78002C1FD198222100520028002D
:10A7F00001F02AFA0123C420FF222B700C4B8000A9
:10A800001C635C630B4B1C605C600B4B19589143E1
:10A810003F3A0A431A50802252021A600D20074A1A
:10A82000074900F0F1FF200070BDC046FC65FF1F26
:10A8300000800040A0F0004000E100E0ADA6001163
:10A84000ADA40011030010B50620072B09D8054A56
:10A85000137001F061F9D7210020034B034A8900EE
:10A860005A5010BD5043FF1F0000FF1F8D1BFF1FDC
:10A8700070B51D0002240C2910D8094ACA40D2071D
:10A880000CD5FBF72FFF041E08D1059A0499280068
:10A89000FBF744FFFCF7B2FDFFF712FB200070BD91
:10A8A0001210000030B50D7802232C009C43184292
:10A8B00001D02B431C0008252300AB43284201D0C4
:10A8C0002B00234320241D00A543204201D01C431C
:10A8D00025002A230D70184204D011781E3B0B432B
:10A8E000137030BD0028FCD10C2113788B43F7E79F
:10A8F000F8B51D0006AB1B88140007AA0E000B203C
:10A900001778002B27D10A78022A49D14A68507853
:10A9100011780002244A08438018042840D800F027
:10A92000B3FF03121D1B2300F06801F0BDF9021CE8
:10A93000C0B2B84200D93A1CD2B22000F1682A80D5
:10A9400000F00AFF06E00222F3681B882A802370C9
:10A950001B0A63700020F8BD0622EEE701232B805E
:10A96000F3681B782370F5E7F368002B16D00822F4
:10A970002A801A8822701A88120A62705A88A27075
:10A980005A88120AE2709A8822719A88120A6271B1
:10A99000DA88A271DB881B0AE371DBE72B80D9E739
:10A9A00001202B80D7E7C04600D6FFFFF7B5160081
:10A9B0000A781D0008AB1F880C000123022A18D159
:10A9C0004A685078117800022B4A084380180328FF
:10A9D0000FD800F059FF02254439E06801F064F90E
:10A9E000C0B20723B84204D37B190193152B02DDB3
:10A9F0000D231800FEBDE0682A003100C01900F0E8
:10AA0000ABFE6B4600209B88E268D0541B4B1B6852
:10AA1000834203D01B68834200D098470023E8E7B5
:10AA20000B23002FE5D1022DE2D1737832781B027F
:10AA30001343E2681380114B1B68002BEED01B6898
:10AA4000002BEBD00120E8E70B23002FD1D1062DFE
:10AA5000CED12A003100E06800F07EFEDEE70B2355
:10AA6000002FC6D1012DC3D132787533012AC0D849
:10AA7000E3681A70D2E7C04600D6FFFF0868FF1FE0
:10AA800070B50C001500072837D800F0FDFE04143F
:10AA900036361B36242E182015290BD8184E1622B0
:10AAA0000021300000F0D8FF22002900300000F023
:10AAB00053FE002070BD18200229FBD11288114BD3
:10AAC0001A80F6E718200829F4D10A000E48290058
:10AAD00001F01AF9EDE718200129EBD10B4B1078A2
:10AAE0000B49DA69FFF7DEFEE3E718200129E1D11F
:10AAF000064B10780749DA6BF4E70220DAE7C04624
:10AB0000F067FF1FCE43FF1FC443FF1F5443FF1FC7
:10AB10007C43FF1F9C43FF1F030010B50020DB0791
:10AB200004D50721024A034800F08CF810BDC04646
:10AB3000A8C000115443FF1F054A030010680028F5
:10AB400003D082889A4201D1806870470068F6E796
:10AB5000006AFF1F0A88030008009A4204D08A880E
:10AB600004309A4200D0002070470000F8B5F2226D
:10AB700000230D4F0D4E7968050042433370994212
:10AB800000D07B600A4C0021200000F065FF00230C
:10AB90001A007C60AB4202D100203370F8BD013353
:10ABA0002280DBB2F234F5E7F86AFF1FF66AFF1F76
:10ABB000046AFF1F73B56B460190060068461500D6
:10ABC0001980FCF74DFF041E11D1002D0FD076899E
:10ABD000002E11D00C2001F00FF800280ED0084AEA
:10ABE0000460136886808560002B02D1106020000D
:10ABF00076BD1A001B68F7E70224F8E71324F6E78E
:10AC0000006AFF1F012100220A4B10B549420A4C7D
:10AC1000198099809A719A70084B207001201980D0
:10AC20005A60FFF7A3FF2078FCF778FF0448FDF790
:10AC300033FF10BD1068FF1F006BFF1FF86AFF1F76
:10AC4000F1AC0011022310B5002802D0FFF7B2FFCB
:10AC50000300180010BD0000030010B50020DB0742
:10AC600004D50421024A0348FFF7A4FF10BDC046E3
:10AC7000BCC00011D443FF1FF0B50E2687B003936C
:10AC80000CAB1F8802ABF6180500080031000292D9
:10AC9000FDF768F804000120002C0FD03088FFF782
:10ACA0004BFF03000E20002B08D05E68002E05D05D
:10ACB00021002800039B029A0097B04707B0F0BD1F
:10ACC0000A4B10B5984207D10122002352420A8054
:10ACD0008B708A808B7110BDFFF73CFF0028FAD083
:10ACE00001235B42038000238370F4E7FFFF000031
:10ACF000F8B5050001290AD1134E00243388F22744
:10AD0000AB4219D028001149FFF7DAFF06E002290B
:10AD100004D10139FDF73EFF0028EDD0F8BD3B001E
:10AD200063437268D018D35A002B09D03A0000212F
:10AD300000F092FE0134E4B2054B1B78A342EED83A
:10AD400001235B423380DDE7F86AFF1F1068FF1FB5
:10AD5000F66AFF1F10B5FFF7FDFE030000208342D7
:10AD600000D0987810BD0000F0B589B01C000EAB83
:10AD700080CB03901E8810AB1B78049202930B7A51
:10AD80000D00DB0616D42B780593022B24D00498F3
:10AD9000FFF7D2FE002812D003689C46002B0ED08D
:10ADA000029B2200019329003B0064460398009611
:10ADB000A04705E00498FFF7BFFE002802D10E204F
:10ADC00009B0F0BD8368002BF9D00A22290003984E
:10ADD00098470028D7D0F3E76B6858781A786B4B00
:10ADE000000210439842D2D8043B984210D2684BDC
:10ADF000984242D015D8674BC0180128C7D80B20FD
:10AE0000002EDDD1EB681A7859683A80200028E0DE
:10AE1000614BC018032800D979E000F035FD846A41
:10AE2000789E5E4B9842B2D10B20002EC8D10123F0
:10AE30003B80EB6831001B7823706889013080B259
:10AE4000FCF790FF3A88031E0ED0017802328A1870
:10AE50003A80428962704289120AA2705968027867
:10AE6000E01C00F079FC06E004323A803100042254
:10AE7000601C00F0F1FD0020A2E70B20002E9FD106
:10AE8000EB6807A91E8804233B80330A3000267034
:10AE90006370FCF767FF051E28D004AB9A890E2368
:10AEA00004A95B183E49C668FCF7D0FF00280BD107
:10AEB0002B783C486A680599FBF786FB002803D18C
:10AEC000012304AA5B42D3813278022A06D1716839
:10AED000201D00F041FC3B8802333B800E2304AA76
:10AEE0009B181B88A3701B0AE370C4E704ABDE81C8
:10AEF000F4E70B20002E00D062E7E9680398FFF723
:10AF000029FF02233B802070000A6070B3E70B200A
:10AF1000002E00D054E70222EB681B883A80237091
:10AF20001B0A6370A7E7E86800F0BEFEC2B2030028
:10AF30000720B24200D243E70DD00299DBB271186C
:10AF4000994202DB921BD3B20293029BE9681A007A
:10AF50003B8089195AE70023F6E70B20002E00D02A
:10AF60002EE70722EB683A801A7822705A786270CE
:10AF70005A88A2705A88120AE2701A792271DA8805
:10AF80006271DB881B0AA37175E7C04604290000C3
:10AF90000228000000D8FFFFFFD6FFFF03280000B3
:10AFA000FFFF0000ECBF0011F0B58DB06B46002034
:10AFB000089120229B5E83423DDAA64B187800F070
:10AFC000FBFC071E32D00378B02B2CD1007902385D
:10AFD00016281FD800F0D0FE17001E001E001E000D
:10AFE00031001E0096001E001D011E0052011E00B1
:10AFF00073011E00CD011E0050021E001E001E0027
:10B000008E021E00E302944B94491B8878880B80C3
:10B01000FBF71AF83800FCF79BFF914B1B68002BDD
:10B0200001D038009847380000F08EFD8020089B42
:10B030000002434018000DB0F0BDEE220021874809
:10B0400000F00AFD0BAA3B7B7989388900923A000F
:10B050000D32FCF79FFD0400804B1B78002C3FD184
:10B0600046E0804B788805937F4B4100CB5A0BAE6E
:10B07000073BDBB232880293002301937B4B210014
:10B0800006930093059BFFF76FFE744D002810D1C7
:10B09000069B3A8A1B889A420BD1380005991230D8
:10B0A00000F0E2FB002804D02B7862899B00EB18AB
:10B0B0005A80162306A81B18328820007989FCF7CD
:10B0C000C5FE2B7804009A00AA1851880029C3D025
:10B0D0000133DBB22B70002807D006A9C98A918002
:10B0E000634A12889A42BCD802E001214942918009
:10B0F000002B04D059497888FAF7DAFF8AE73E89AD
:10B100000A2479E000253E89574B06937B88069AEE
:10B110005B009B5A033B9D4202DB002DF0D05BE0BD
:10B12000162206A812183B7B798900923A0030005B
:10B130000D32FCF72FFD0590002858D04689017A82
:10B140007888FCF7F1FC041E44D1464B78880793BD
:10B15000069B4100C95A454B0439C9B206AAD28A96
:10B1600006930291019400930599079BFFF7FCFD5C
:10B17000041E2FD1069B39491A88931C002D26D115
:10B180004B807988384B4900CB5A5119033B8B428D
:10B1900020DD059B31485B8941190B71A91C0135E4
:10B1A000C9B2EDB2059145191B0A2B71059B2D49BA
:10B1B0000433181800F0D0FA2C4B059A1B88D318CA
:10B1C000DDB22C4B9E4205D00136B6B29CE74988D1
:10B1D0009942D6D0002D0CD0204C2800618800F078
:10B1E000EBFC207021007888FAF772FF12E7059CCB
:10B1F000F0E7002C00D183E77B78142B00D109E71E
:10B2000016493B794E800B700C717888FAF712FF63
:10B2100000E7162406ABE41821003889FCF7A2FDEC
:10B22000011E00D1B7E1788822880F4C45002C5BC5
:10B230000A4D013CE4B2029400240F4B01940095A6
:10B24000FFF792FD041E00D014E129007888FAF778
:10B250004FFFDFE6006BFF1FC042FF1F1868FF1F94
:10B260000C68FF1F0C69FF1F4864FF1FFC69FF1F6C
:10B27000BE42FF1FFFFF00001A68FF1F162406AB27
:10B28000E41821003889FCF76DFD011E00D182E130
:10B2900078882288AE4C45002C5BAE4D013CE4B270
:10B2A00002947C89AC4B01940095FFF75DFD041E70
:10B2B00000D0DFE029007888FAF724FFAAE600250D
:10B2C000A44B1D803B00F6331B78A24A7888079276
:10B2D000AB4208D99E4B12880693069943005B5AED
:10B2E000013B9A4203DB0799FAF716FF92E6162410
:10B2F0006B00FB18059306ABE418059B2100188929
:10B30000FCF730FD011E03D1059B01241E8973E764
:10B310007888924B2288069C099343001B5B904ED1
:10B32000013BDBB20293002300960193099BFFF7D8
:10B330001BFD041E02D0059B1E895DE77B88069AD3
:10B340005B009B5A079A108832881218934202DCDD
:10B350001B1A013B33807F4C023032880999001957
:10B3600000F0FAF92388328801359B182380EDB26A
:10B37000A8E70BAA3B7B7989388900923A000D3205
:10B38000FCF708FC00250590059B002B04D10A243E
:10B39000002D00D16EE060E0059B7888197AFCF7FB
:10B3A000C3FB0100041E63D1694C6C4B7888069482
:10B3B0000993069B4400E45A694B063CE4B20BAE89
:10B3C000328807930294019100930599099BFFF736
:10B3D000CBFC041E4CD1079B5E491B881A1D002D17
:10B3E00030D14A80059B5B4C5A8963191A716B1CDA
:10B3F0009BB2E318120A1A71162306A832881B188A
:10B4000079890598FCF722FDFF21AA1C2E1D033522
:10B410000B00059092B2B6B2ADB2002803D006ABD5
:10B42000DB8AD9B21B0AA218651911712B714C4D18
:10B43000301D2A884949201800F08EF92B88F6180B
:10B44000B5B2A1E74988914207D17A88069952009E
:10B45000525AEB18053A9A42C4DC3E4C28006188E7
:10B4600000F002FC207021007888FAF75FFED1E539
:10B47000002DF2D13E89BFE6162606ABF618310044
:10B480003889FCF76FFC3D000400FA3500282DD008
:10B49000037A9B060CD400227B8939897888009234
:10B4A0003A000C32FFF7E8FB041E10D03E8915E08D
:10B4B0003088FFF741FB00281AD08368002B17D093
:10B4C0002100122278889847041EE4D0EEE72B78FA
:10B4D000002B02D17888FAF739FE00262B78002B52
:10B4E00000D097E5002C00D194E585E60124DDE746
:10B4F0000E24DBE7162506ABED1829003889FCF78A
:10B5000031FC041E47D0037A9B0611D4154A7B8870
:10B510001188994203D01448814207D11380134BFC
:10B52000F2261D780023D9B2A94221D30924A1E72C
:10B530002888FFF701FB00282FD08368002B2CD030
:10B540002100122278889847041EDFD092E7C04677
:10B550004864FF1F1868FF1F1A68FF1F0C69FF1F50
:10B56000FC69FF1FF86AFF1FFFFF0000F66AFF1F5C
:10B5700031005943546801336018615A0029D2D10F
:10B580003C0008342100F22200F0E6F8210078881F
:10B59000FAF7E4FD3EE501246CE70E246AE71D4B53
:10B5A0001A887B889A4231D07888FAF7E1FD31E534
:10B5B000F223059851684343CD18C95A00291FD07A
:10B5C0003B7A012B0BD16C88AB887888AA1D00943C
:10B5D000FFF752FB041E02D000233B722E88F2229A
:10B5E0000021280000F038FA00232B80059B01334E
:10B5F000DBB20593084B05991B78064A8B42D7D8D6
:10B6000001235B421380002CCED0F5E500263400E8
:10B610000596EFE7F86AFF1FF66AFF1F70B5040092
:10B620000E001500FFF796FA031E08D131000548F9
:10B63000FFF790FA03001120002B02D01C8000209D
:10B640009D7070BDFFFF0000F8B50B4F06003B7802
:10B650000D001400FF2B0ED00A2000F0C5F9011ECA
:10B6600009D0B1230380002346800371C580048183
:10B67000387800F061FBF8BD1544FF1FF7B50F00E7
:10B6800008A90600088809A90B240988002821D1E7
:10B690000234022B1ED1557813782D021D432B0046
:10B6A0008B4301937334002B14D1FB6830001900D5
:10B6B0000093FFF74FFB019C85420BD02A0030001E
:10B6C0000099FFF7ABFF041E04D12A0030007989EE
:10B6D000FFF7BAFF2000FEBDF0B50E7885B00390ED
:10B6E0000AA805880120022E0DD14C6827786478BD
:10B6F00024023C43054FBC4205D10398DBB20196BE
:10B700000095FFF7BBFF05B0F0BDC0460229000061
:10B71000034B10B51B68002B00D09847FEE7C046CE
:10B72000046BFF1F07B501A8FFF7F2FF044A0548A5
:10B730000021121A00F088FAF8F79EF8FEE7C046DA
:10B74000086BFF1F1844FF1F01B40248844601BC68
:10B75000604700BFAD32FF1F01B40248844601BC00
:10B76000604700BFE94C010001B40248844601BCB7
:10B77000604700BFADAE000001B40248844601BC82
:10B78000604700BF0519FF1F01B40248844601BC91
:10B79000604700BF3D36FF1F01B40248844601BC2C
:10B7A000604700BFC926000001B40248844601BCBE
:10B7B000604700BF5549010001B40248844601BCFE
:10B7C000604700BF1D3AFF1F01B40248844601BC18
:10B7D000604700BF6D30FF1F01B40248844601BCC2
:10B7E000604700BFA54F010001B40248844601BC78
:10B7F000604700BF2526000001B40248844601BC12
:10B80000604700BF851F000001B40248844601BCA8
:10B81000604700BF0D31FF1F01B40248844601BCE0
:10B82000604700BF8530FF1F01B40248844601BC59
:10B83000604700BF1D4B010001B40248844601BCB3
:10B84000604700BF3119FF1F01B40248844601BCA4
:10B85000604700BFC9A9000001B40248844601BC8A
:10B86000604700BF8D12000001B40248844601BC4D
:10B87000604700BFCD4C010001B40248844601BCC2
:10B88000604700BFE548000001B40248844601BC9F
:10B89000604700BF1D3BFF1F01B40248844601BC46
:10B8A000604700BF0D52010001B40248844601BC4C
:10B8B000604700BF2951010001B40248844601BC21
:10B8C000604700BF6571010001B40248844601BCB5
:10B8D000604700BF156B010001B40248844601BCFB
:10B8E000604700BFF938FF1F01B40248844601BC1D
:10B8F000604700BFD91B000001B40248844601BC68
:10B90000604700BF4936FF1F01B40248844601BCAE
:10B91000604700BF3D37FF1F01B40248844601BCA9
:10B92000604700BF6DBC000001B40248844601BC02
:10B93000604700BF4D1F000001B40248844601BCAF
:10B94000604700BFF30E000001B40248844601BC0A
:10B95000604700BFE538FF1F01B40248844601BCC0
:10B96000604700BF3D18000001B40248844601BC96
:10B97000604700BFE117000001B40248844601BCE3
:10B98000604700BFED4A010001B40248844601BC93
:10B99000604700BF5147010001B40248844601BC22
:10B9A000604700BF055E000001B40248844601BC48
:10B9B000604700BFB139FF1F01B40248844601BC93
:10B9C000604700BFF54E010001B40248844601BC47
:10B9D000604700BF75A9000001B40248844601BC5D
:10B9E000604700BFF137FF1F01B40248844601BC25
:10B9F000604700BF1D4D010001B40248844601BCF0
:10BA0000604700BFC94A010001B40248844601BC36
:10BA1000604700BF691F000001B40248844601BCB2
:10BA2000604700BF7139FF1F01B40248844601BC62
:10BA3000604700BF1147010001B40248844601BCC1
:10BA4000604700BFC53AFF1F01B40248844601BCED
:10BA5000604700BF9DA9000001B40248844601BCB4
:10BA6000604700BF154D010001B40248844601BC87
:10BA7000604700BF091B000001B40248844601BCB6
:10BA8000604700BFE928000001B40248844601BCB9
:10BA9000604700BF093BFF1F01B40248844601BC58
:10BAA000604700BFC521000001B40248844601BCC4
:10BAB000604700BF8552010001B40248844601BCC2
:10BAC000604700BFC56D010001B40248844601BC57
:10BAD000604700BF7918000001B40248844601BCE9
:10BAE000604700BF014C010001B40248844601BC1C
:10BAF000604700BFED3AFF1F01B40248844601BC15
:10BB0000604700BF5D17000001B40248844601BCD5
:10BB1000604700BFDD66010001B40248844601BCF5
:10BB2000604700BF8D1BFF1F01B40248844601BC63
:10BB3000604700BFC51D000001B40248844601BC37
:10BB4000604700BF0534FF1F01B40248844601BCB2
:10BB5000604700BF434D010001B40248844601BC68
:10BB6000604700BFB54C010001B40248844601BCE7
:10BB7000604700BFB14E000001B40248844601BCDA
:10BB8000604700BF2124000001B40248844601BC84
:10BB9000604700BF291C000001B40248844601BC74
:10BBA000604700BF6D36FF1F01B40248844601BCE8
:10BBB000604700BF8B52010001B40248844601BCBB
:10BBC000604700BF350E000001B40248844601BC46
:10BBD000604700BF4551010001B40248844601BCE2
:10BBE000604700BFD949010001B40248844601BC46
:10BBF000604700BF017F000001B40248844601BCD9
:10BC0000604700BF3D4B010001B40248844601BCBF
:10BC1000604700BF5952010001B40248844601BC8C
:10BC2000604700BF056A000001B40248844601BCB9
:10BC3000604700BF350E000001B40248844601BCD5
:10BC4000604700BF4550000001B40248844601BC73
:10BC5000604700BFB70E000001B40248844601BC33
:10BC6000604700BFF94C010001B40248844601BCA2
:10BC7000604700BF090E000001B40248844601BCC1
:10BC8000604700BFD532FF1F01B40248844601BCA3
:10BC9000604700BFB352010001B40248844601BCB2
:10BCA000604700BF3139FF1F01B40248844601BC20
:10BCB000604700BFDD52010001B40248844601BC68
:10BCC000604700BFA946010001B40248844601BC98
:10BCD000604700BF090E000001B40248844601BC61
:10BCE000604700BF3555000001B40248844601BCDE
:10BCF000604700BF0124000001B40248844601BC33
:10BD0000604700BF993AFF1F01B40248844601BC56
:10BD1000604700BF810E000001B40248844601BCA8
:10BD2000604700BF2146010001B40248844601BCBF
:10BD3000604700BF2D2EFF1F01B40248844601BC9E
:10BD4000604700BF594F010001B40248844601BC5E
:10BD5000604700BF5125000001B40248844601BC81
:10BD6000604700BF311B000001B40248844601BC9B
:10BD7000604700BF456B010001B40248844601BC26
:10BD8000604700BF313BFF1F01B40248844601BC3D
:10BD9000604700BFEDA5000001B40248844601BC25
:08BDA000604700BF55220000BE
:10BDA800000101030200030304030502060207025F
:10BDB800080209020A030B030C020D000E030F030D
:10BDC800100311001300140315001600313C001174
:10BDD800653C00110000000002000000EABD0011EF
:10BDE800192A0F180A000000F1590000FD2400006C
:10BDF80041460100A1810011B5A100110976001189
:10BE0800A57F001135540011A9AF00118150001110
:10BE1800413E0011713F001100000000161600009D
:10BE28000200000034BE0011F4FFF3FFD2FC000052
:10BE3800B140001100000000000000005475796155
:10BE48000042312E39003030313900676974687525
:10BE5800622E636F6D2F70767678005448303546C1
:10BE6800000000000200000080BE0011292A282AD4
:10BE7800272A262A252A242A0A180000E204000074
:10BE88007102000078EC000005000000744000001A
:10BE98001027000060F000000400000006640000A5
:10BEA800204E000000000000060000005C44000076
:10BEB800102700006CEE00000700000005000000DD
:10BEC8001F501D00023CB4000001190019000000B9
:10BED800A102000030313233343536373839414227
:10BEE8004344454600000000395800118D580011A0
:10BEF800000000000200000008BF00116F2A6E2A2F
:10BF08001A18EAD8BC80F0FC6000000000000000AD
:10BF1800000000F505D39727B6F615F7B777E6F0D2
:10BF2800C7F27200000001A0000000006410B71DF5
:10BF3800C8206E3BAC30D9269041DC76F4516B6B4F
:10BF48005861B24D3C7105502083B8ED44930FF011
:10BF5800E8A3D6D68CB361CBB0C2649BD4D2D386C7
:10BF680078E20AA01CF2BDBDFB349B5F8000008014
:10BF780000100000000000000B620011957800110D
:10BF88002F6200119D7C0011B3620011737C0011B7
:10BF980029630011497C00117B630011117E001197
:10BFA800E3630011117E001115640011CB7D0011AF
:10BFB80029630011017C0011A1630011A97D001102
:10BFC800000000000000000087640011A97D001136
:10BFD800E9640011AD780011052A042A012A002A13
:10BFE8000229032801280028011800180000000071
:10BFF80000000000000000000000008701010201AD
:10C00800020101020102030304010301010101010C
:10C018000303020103000D000E00100011001300BD
:10C028001401070108010A010B011C011D02040289
:10C0380005020702080219021A021C021D03010365
:10C04800020317000201000504000807000B0A009C
:10C058001716001D1C010201010504010E0D011136
:10C0680010011413011716011A19020201020B0A12
:10C07800020E0D0211100214130217160305040311
:10C088000807030B0A030E0D0001020307090A0B38
:10C098000E0F101112141718191A1B1F2021220035
:10C0A800F1A80011ADA90011000000000200000075
:10C0B800F2BF001100000000D9B600110000000016
:08C0C80002000000F0BF0011AE
:020000041FFFDC
:1000000000000000A93D0011F0BD0011ECBD001181
:100010004861FF1F00000000000000000000000019
:1000200000000000000000000000000000000000D0
:1000300000000000000000000000000000000000C0
:1000400000000000000000000000000000000000B0
:1000500000000000000000000000000000000000A0
:100060000000000000000000000000000000000090
:100070000000000000000000000000000000000080
:100080000000000000000000000000000000000070
:100090000000000000000000000000000000000060
:1000A0000000000000000000000000000000000050
:1000B0000000000000000000000000000000000040
:1000C0000000000000000000000000000000000030
:1000D0000000000000000000000000000000000020
:1000E0000000000000000000000000000000000010
:1000F0000000000000000000000000000000000000
:1001000000000000000000000000000000000000EF
:1001100000000000000000000000000000000000DF
:1001200000000000000000000000000000000000CF
:1001300000000000000000000000000000000000BF
:1001400000000000000000000000000000000000AF
:10015000000000000000000000000000000000009F
:10016000000000000000000000000000000000008F
:10017000000000000000000000000000000000007F
:10018000000000000000000000000000000000006F
:10019000F932FF1F5931FF1FC16601000000000046
:1001A000000000000000000000000000000000004F
:1001B000000000000000000000000000000000003F
:1001C000000000000000000000000000000000002F
:1001D000000000000000000000000000000000001F
:1001E000000000000000000000000000000000000F
:1001F00000000000000000000000000000000000FF
:1002000000000000000000000000000000000000EE
:1002100000000000000000000000000000000000DE
:1002200000000000000000000000000000000000CE
:1002300000000000000000000000000000000000BE
:1002400000000000000000000000000000000000AE
:10025000000000000000000000000000000000009E
:10026000000000000000000000000000000000008E
:10027000000000000000000000000000000000007E
:10028000000000000000000000000000000000006E
:10029000000000000000000000000000000000005E
:1002A000000000000000000000000000000000004E
:1002B000000000000000000000000000000000003E
:1002C000000000000000000000000000000000002E
:1002D000000000000000000000000000000000001E
:1002E000000000000000000000000000000000000E
:1002F00000000000000000000000000000000000FE
:1003000000000000000000000000000000000000ED
:1003100000000000000000000000000000000000DD
:1003200000000000000000000000000000000000CD
:1003300000000000000000000000000000000000BD
:1003400000000000000000000000000000000000AD
:10035000000000000000000000000000000000009D
:10036000000000000000000000000000000000008D
:1003700025B7001100000000000000000000000090
:10038000000000000000000000000000000000006D
:10039000000000000000000000000000000000005D
:1003A0000000000000000000000000000D1BFF1F07
:1003B000000000000000000000000000000000003D
:1003C000000000000000000000000000000000002D
:1003D000000000000000000000000000000000001D
:1003E000000000000000000000000000000000000D
:1003F00000000000000000000000000000000000FD
:08183800106FFF1F4118FF1F94
:10184000024981F3088802F0C7FB0000106FFF1FF8
:1018500070B500241E491F4A1F484C6308CA1B0567
:101860001B0DE4188242F9D11C4B80228B630021AE
:1018700009201B4B920519621A4B1B4DDA671B4B53
:10188000DA688243DA609A68194802409A60112047
:10189000296002F08DF8112002F06AF880226B6C4A
:1018A000112093436B64EE23DB006343114A1B0C4E
:1018B00013840122104B9A7201F004FC0F4B1B7829
:1018C000002B04D10E4B1021187802F08DFB70BD57
:1018D000000005408805054000060540FF010000A6
:1018E00000F0004004E100E0003800403CF000401F
:1018F000FFDFFFFF1861FF1FCC61FF1FFA63FF1FAF
:10190000F861FF1F10B502F037F9072804D012283C
:1019100008D0022808D010BD044A0420136B0133FC
:101920001363F8E70220F6E71420F4E7F064FF1FE2
:10193000F8B507000C0026002500503630785135E8
:10194000002804D10300287058342370F8BD29788A
:10195000CA00481E8141A3183800A25C5B68C9B266
:10196000FFF7D0FF00280DD12B78DA00A218013341
:1019700050602B703378044A013B3370136A013393
:101980001362D8E70123DFE7F064FF1F5C234343C2
:10199000074910B5C9180B0058331B78012B05D126
:1019A000FFF7C6FF034A936A0133936210BDC04636
:1019B0002465FF1FF064FF1F10B502F0CDF8064A42
:1019C0000121130010CB4942D967044B136002F088
:1019D000D3F9200010BDC04600E100E01000100067
:1019E00010B5040002F0B8F8024B1C6002F0C4F914
:1019F00010BDC04600E100E0431E5A425341A02200
:101A0000F0B5D2015B421340154D164A40019B18B8
:101A10002A18127E8BB00191002A1BD01A000832BE
:101A2000D46F0022E6B206AFE4B294420EDC28186E
:101A3000C369002B08D0019902AA117106AA049269
:101A400002AA167303A898470BB0F0BD1978B954D1
:101A50000132EAE71A7D1A7806AB01261A70E6E72A
:101A6000B067FF1F00400040F0B5254B0400400167
:101A7000C25C85B0002A2BD01A18117E002927D00D
:101A8000917E002924D01179022921D11689D78885
:101A9000D168F51BADB22A1C102D00D9102292B2CC
:101AA000BE4217D11818012303710023C269C380F5
:101AB00003819A4206D068460321037301710293A1
:101AC00001A890470820002C00D0192001F0FAFA54
:101AD00005B0F0BD013C65426C41A0256442ED01BA
:101AE0002C40084D1B186419074D0633013A92B279
:101AF000AA42EDD01888461C1E80085C2070F5E7CD
:101B0000B067FF1F00400040FFFF00000F220E4B98
:101B100010B59868104002380A280BD801F0FEFF73
:101B20000D0A0B0A0A110A0A0A0A060002210020FD
:101B3000FFF762FF10BD0121F9E70020FFF794FFD6
:101B4000F8E7DB6FF6E7C046004000400F220E4B7F
:101B500010B59868104002380A280BD801F0DEFF53
:101B60000E0A0B0A0A120A0A0A0A060002210120BA
:101B7000FFF742FF10BD01210800F9E70120FFF740
:101B800073FFF7E7DB6FF5E70090004013B5334CC8
:101B90002378072B3DD8324B1A78324B002A39D1A3
:101BA0008022196852020A431A60252001F0C0FE03
:101BB00020232D4A11680B43802113606B460422B9
:101BC000C90508680733104228D080210422C905BE
:101BD000C86810422ED080212020C905CA688243DF
:101BE000CA6014221A701A78002A2FD18021C905E0
:101BF000C86820320243CA6014221A701A78002A78
:101C000028D11A4B1A7D22785A601D221A70593237
:101C1000DA6013BD1A6816490A40C5E7086802432E
:101C20000A6014221A701A78002ACED01A78013A63
:101C3000D2B2F7E7C8680243CA6014221A70197852
:101C40004A1ED2B21A700029F9D1C4E71A78013AB3
:101C5000D2B2C7E71A78013AD2B2CEE75043FF1F9B
:101C60001844FF1F3CF000404843FF1F0020004085
:101C7000FFFFFEFF564B70B51B68012B03D1554A81
:101C8000936D0133936501F0DFFF534B534A1860A6
:101C9000534B544C1A600123534A1360534A136048
:101CA0002378002B06D006225149524802F0D4F87E
:101CB00000232370504A514B10681B78C1B2002B8F
:101CC0000ED14F4CC0B223785BB2002B4FDB237890
:101CD00024785BB264B21B0424021B191B18136026
:101CE0000B1C50294ED95023464A47491078DBB285
:101CF000FF2202284BD10868444C454D267890437A
:101D00002A78964254D9227824782E78023B5D10A6
:101D1000A31B6B435201D31A10335B1118430860A5
:101D200002F0DAF8031F012B45D83A4B1B78002B41
:101D300006D0394B1B78002B02D0002001F014FF95
:101D4000A122364B92009978354B4A431B689B1869
:101D5000832292009B181B78033B012B03D8AF20F2
:101D6000400002F0E9F801222E4BDA8270BD2378A0
:101D700024785BB264B2FF33FF341B0424021B19C6
:101D80000138ABE7CAB2022AAED20223ACE7086838
:101D9000254C264D267890432A78964208D92278F9
:101DA00024782D78023B5B10641B63435201B2E739
:101DB0002378DBB2B2E70228D5D11D4B1B78013B5B
:101DC000022B03D91B4B1B78022BCCD16C20C8E70C
:101DD0009809FF1FFC0FFF1F3C64FF1FFF3F00001F
:101DE000141003404064FF1F0C1003400010034018
:101DF000D50BFF1F7211FF1FB40003408C09FF1F9A
:101E0000680AFF1F490AFF1F94000340460AFF1F8C
:101E1000470AFF1FF908FF1F2209FF1F300DFF1F90
:101E20003409FF1FBC0BFF1F440AFF1F450AFF1F99
:101E30001C09FF1F2309FF1F10B501F08DFF0022B1
:101E4000014B1A8010BDC0463A64FF1F10B502F066
:101E5000D3F8A121054A89009478054A61431268A4
:101E6000044B5218528C1A8010BDC046300DFF1F13
:101E70003409FF1F3A64FF1F10B50D4B0D4A9978C6
:101E8000A1239B004B431268D218531DD97F0A4BE4
:101E90001B88994209D2441C07D0C82805D0D269B2
:101EA0005B1A5A43054B5343C01801F02DFF10BD78
:101EB000300DFF1F3409FF1F3A64FF1F710200003D
:101EC00070B5244D2B68002B28D002F09DF82B68AC
:101ED000D8402B680400002B27D001F075FF2B6839
:101EE000D8401D4B1D4A9978A1239B004B43126893
:101EF000D118D25C91239B00002A20D0CA5801320D
:101F0000CA50174B17491B680868834214D3D23B49
:101F1000181A012A1AD0144B186070BD02F074F818
:101F2000124B196801F090FFD3E701F04DFF0F4B02
:101F3000196801F089FFD4E70D495B18E8E7CA503A
:101F40000C4B1B68DB68E418201AE4E7F530FF301F
:101F5000E1E7C0461C08FF1F300DFF1F3409FF1FBB
:101F60009C09FF1F3C64FF1FA009FF1F1808FF1FEB
:101F70002DFF3F004464FF1F70B504000D002829A9
:101F800016D10300A433C2881B889B1A0B4A9BB24C
:101F900093420DD906006A3605223100653001F002
:101FA00023FE002804D13100200001F09DFF70BD08
:101FB0002900200002F038F8F9E7C046FE7F000053
:101FC000F8B50500012001F01FFE134CA36AA26AB8
:101FD0009342FBD1114E336001F04EFF10490300D4
:101FE00008601048426894460F4A17680022BC45B2
:101FF00001D24268BA1A0D4802603268AD18A422B4
:10200000E562606A520302436262094A1278002A5A
:1020100001D00F3B0B60F8BD00F00040340AFF1FF9
:10202000E408FF1F28100040180AFF1F1C0AFF1FAA
:102030001C09FF1F70B580241025E405A3682B43FD
:10204000A36001F0F1FDA368AB43A36070BD000085
:10205000F7B5160080221C001023D205019191686B
:1020600005000B43936000225A4BD7301A6001F0F1
:10207000E3FE9D232A002F009B00EB58CA3201216A
:102080000092FC37002B01D00021009A386801F043
:10209000FBFD2900009BCB311A784F4BD3351A60DA
:1020A0004B780A781B0213438A7812041A43CB78C0
:1020B0001B061343494A1BBA13604B790A791B026A
:1020C00013438A7912041A43CB7931001B06134358
:1020D000434A1BBA13606B782A781B021343AA7811
:1020E00012041A43EB781B0613433E4A1BBA1360D3
:1020F000019A330213433C4A13603C4B22001B1BE2
:102100009C4603293DDCB3089A0013005142B21AE1
:10211000032A46D1354AE018511A827840781204D1
:1021200000020243E05C043302430A600022FF2BFA
:102130004BDDF0222E4B12011A600F222D4B1A603C
:102140002D4A1368002BFCD00023224A2749136034
:10215000091B321D0B191B68043A180A23706070A2
:10216000180C1B0EA070E3700434002AF2DC8022ED
:1021700010213B68D20501333B6093688B43936029
:10218000F7BD6346D578981893782D061B042B432A
:10219000157804392B43557804322D022B43036004
:1021A000AFE7022A0AD1114AE05C511AE2185278CC
:1021B000120202430A6004339BB2B7E7012AB5D189
:1021C0000A4A521AE15C1160F5E7084959180A6099
:1021D0000433ACE7000004403C00044038000440F5
:1021E00034000440300004400C000440000104406E
:1021F000040004401000044014000440F7B515002A
:1022000080221C001023D2050091916807000B4327
:1022100093600023654AD730136001F00DFE9D23C3
:102220003E009B00F9583B00CA363200FC330029BF
:1022300000D07FE0586801F027FD390032785C4B10
:10224000CB311A604B780A781B0213438A78AC466C
:1022500012041A43CB78281D1B061343554A1BBA98
:1022600013604B790A791B0213438A7912041A43CB
:10227000CB791B061343504A1BBA13604B7A0A7A78
:102280001B0213438A7A12041A43CB7A21001B06DD
:1022900013434A4A1BBA1360009A2B021343484A5D
:1022A00013602200474B1B1B0093009BCE785B18EA
:1022B00001938B7836061B0433430E78043833437E
:1022C0004E78043136023343019E33600328ECDC40
:1022D0000321A808431C9B002940800003292BD11F
:1022E0003849E5185E18A9786D78E35C09042D0279
:1022F000294319433160030008330021FF2B2DDDF2
:10230000314B324919600F21314B196001232749A4
:102310000B60304B19680029FCD006211B680B406C
:10232000042B20D080220020D20593680A318B43F1
:102330009360FEBD01217DE7022908D121495D1886
:10234000E1184978E35C090219432960D3E70129C0
:10235000D3D11C495918E35C0B60CCE71948181815
:1023600001600433CAE7002310490B606346002B69
:102370000CDC3B00FC335A68102101325A60802289
:10238000D205936801208B439360D2E7009B9B1892
:102390001B68190A13705170190C1B0ED37004239B
:1023A0005B4291709C440432E0E7C0460000044068
:1023B0003C00044038000440340004403000044035
:1023C0000C0004400001044004000440080F000019
:1023D000100004401400044070B5061E19D00222FB
:1023E0005A4B9B799343012B13D1594B1A78FF2AEF
:1023F0000FD15A78FF2A0CD19A78FF2A09D1DA78BE
:10240000FF2A06D11A79FF2A03D15B79FF2B00D16D
:1024100099E0504B0C201A78012A08D000224E4D2A
:102420001A7029780B00093B042B01D8212070BDBC
:102430004B1F012BFAD9454CA37B042B00D982E01A
:10244000A279032A00D97EE09A1ED2B2012A02D8CC
:1024500060881F2877D9002E56D0012E73D1A0880E
:102460000128E3D0002907D1581E032803D801F022
:1024700055FB121715122E702978481E032811D803
:102480000025364B1D602823237501F05DFDA84211
:1024900027D0A580CAE702212970EDE70421FBE7D8
:1024A0000321F9E707390129C0D82D490968C96A0C
:1024B0008906BBD52B4908780028B7D1012A01D954
:1024C000002BB3D102230B708021274D26338901C5
:1024D0002878237501F080FC80212878890101F09B
:1024E00083FD0123A380214B1B78002B0AD0FA2205
:1024F00080211F4B92001B8809025A431A4B1878FF
:1025000001F08AFD002092E701F026FB2B78A680DF
:10251000073B012B03D917482E7001F02DFD114BFD
:10252000114C1A78002A06D08021002220788901D7
:102530001A7001F051FC01F01FFC80212078090283
:1025400001F04AFCDEE7122071E7C046A60BFF1F30
:102550006B09FF1F1A09FF1F1C09FF1F4809FF1FF6
:102560004464FF1F2309FF1F1B09FF1F2109FF1FD1
:102570002C09FF1F0010004010B5002901D001F008
:10258000A3FC10BDF7B5604B01919978A1239B0086
:102590004B435E4A060014681022E418D6235B0001
:1025A000E0583623FF33E35C00279343222B41D1CD
:1025B000574B0F3A1A600760012501F02DFC019B73
:1025C0001880E8235B00E35C002B01D0B34258DDA8
:1025D0000023504FFB70AD33FF33E3581A68002AD5
:1025E00003D09B88DB439B071DD03823FF33E35C7C
:1025F000002B18D09B235B00E35C002B13D1D1335D
:10260000FF33E35CB3420EDAA4235B00E15AE01827
:10261000090A023101F058FB23000122FE33013E7A
:1026200001351A87FA70E8235B00E35C002B2AD09F
:10263000A8B2FEBD03683D00002BBED081880430E7
:10264000090A023101F040FBD6235B00E3581F600A
:10265000B2E72300B133BA00FF33985801378188BD
:102660000430090A023101F02FFBE8235B00E35C30
:10267000BB42EEDCE822F61AED1800235200A35408
:10268000A6E70027F1E7200001F09EFC00281FD0FC
:10269000002E1DDD7319882647190193B60020000E
:1026A00001F0B2FB5A308000201840680135818863
:1026B0000430090A023101F007FB200001F054FB4D
:1026C000A3590133A351BD4202D0019B9D42E6D1E3
:1026D000114BE35C002BABD095239B00E35C002BFC
:1026E000A6D00E4BE15A0029A2D00D4AA35C994214
:1026F00002D90133A3549BE700231A212000A354DD
:1027000001F002FC94E7C046300DFF1F3409FF1FA3
:1027100000140340E010FF1F5A0200007202000084
:102720005E0200000D4970B54A6E0D4CD2038B69F4
:10273000D20BA24206D80B4D0224AA4204D901F0C2
:1027400023FC70BD02246442E21815007E2425405B
:102750002242F4D0A3432B438B61F0E700F000400A
:102760000A200000FC1C0000F8B51D4B1D4F1A7814
:10277000002A10D1BA7B002A02D101321A7003E07C
:10278000032AFAD0022AF8D001F0DEFB0022012051
:10279000154B1A70F8BD154B154D1C68154B9E78DE
:1027A00001232B702878C0B200F09EFBBB7B002B6E
:1027B0000BD101F0F1FAA1239B007343E4188323AA
:1027C0009B00E41823782B70E4E7032B02D101F07F
:1027D00073FBF0E70020022BDCD101F0BDFBEAE740
:1027E0001C09FF1FA60BFF1F2309FF1F3409FF1F32
:1027F000490AFF1F300DFF1FF0B587B00EAD2F78CF
:102800000FAD2D780593AC46634614000E4D0CAA0F
:1028100012782E7803930D9B009201932200059B62
:10282000029701F041FA2E70012C01D0042C08D13E
:10283000802206498B889343054A1278D2011343BC
:102840008B8007B0F0BDC0461C09FF1F6C11FF1F35
:102850007809FF1F0B001B3B70B504003020E02BF4
:102860000DD81300E025493BFF3B9BB2ED00AB4286
:1028700005D8034B200019825A8201F00DFB70BD70
:102880008410FF1F10B501F0DFF9054B00205B68D5
:10289000052B04D9034A5268D20200D4980810BD0F
:1028A00000100040FCE100E070B501F055F90D4B5F
:1028B0001B68FC33DC691D6AFFF7E4FF641984427E
:1028C00004D2094B01241B68002B07D004220024EA
:1028D000064B1A70064A93690133936101F04CFA72
:1028E000200070BD4464FF1F9809FF1F2309FF1FCC
:1028F000FC0FFF1F70B50C4D2B68FC335C6A01F0B8
:102900002BF9FFF7BFFF2B680025FC339B6AE31808
:10291000834204D2054B1B68AB4200D1051B01F07A
:102920002BFA280070BDC0464464FF1F9809FF1FA2
:10293000D722044B92009B5810B5002B00D098472B
:1029400010BDC0460000FF1F10B501F0CFF8FFF723
:10295000EFFF2749274BCA6D274C1A4084235B00A1
:102960001343CB65254B1B68186A01F04DF9244BC6
:10297000244A1A60244B254A1A60A022244B520094
:102980001A60244B187801F01FF92000224901F049
:1029900003F90023A3600233A360204B2049236086
:1029A00003232048A36001F0F7F810221E4BFF20FC
:1029B0001A60802252031A60802292031A608022D9
:1029C00012041A6001F0D0F8012001F085F9FA2014
:1029D000400001F049F9582001F0AEFA134801F027
:1029E000B3F8012001F018F9072001F095FA10BDA5
:1029F00000F0004000FEFEFF141000404464FF1F82
:102A0000000003400180063DBC0003403408000084
:102A1000A40003404A0AFF1F71020000C30900001E
:102A2000FFFF3F002810004000E100E0307500008B
:102A3000674E336888331B6883F3088801F0A4F974
:102A4000644A6549136800200B401360634B644A75
:102A50001B68934200D1A6E001F016FA0221614AF8
:102A600013688B431360FFF76FFF5F4B5F4C187861
:102A7000C0B201F0B1F80023A3600233A3605C4B45
:102A80000120236001F0C0F80323A36001F0B4F932
:102A9000040001F0D9F8050001F0AEF9554B1860BB
:102AA00001F082F8544B1968621A531EA14200D2F9
:102AB00013008022D203934201D39B029B0A326807
:102AC000D16AC90700D471E04C491C0C09689BB25B
:102AD0004C4359432402090A641803264849FC322E
:102AE00093680A6847489B1A474A0768126847492B
:102AF0009B18474A9A1833409208DB190A60036012
:102B0000042B03D9013233400A6003600E68414947
:102B1000A619300001F098F93F4F3E493B68C318B1
:102B20003B603000019301F067F83C4E30680818B4
:102B300038493060884205D9019B01333B6001F080
:102B40005BF8316001F0F0F8354B1B78002B0DD0AD
:102B500001F07AF8334B621B196812188A4232D29C
:102B60004919091B091A304801F016F82F4E337A1B
:102B7000002B0ED001F068F8621BF1681218914228
:102B800024D94919091B091A294801F005F800231D
:102B90003372284B83F3088801F08EF8002001F08F
:102BA00073F901F049F801F06FF95CE7DC01990075
:102BB0000234641A5900641A09214B438033CB4014
:102BC000A408E41889E7FA218900CCE71A49DBE771
:102BD0004464FF1F1CF00040FFFFC1FF0C0AFF1FF1
:102BE000B641210310000040490AFF1F14100040A5
:102BF000C3090000100AFF1F340AFF1F380AFF1F15
:102C0000200AFF1F280AFF1F1C0AFF1F240AFF1F9C
:102C1000C4090000710200006008FF1F2C0AFF1F9A
:102C20001C09FF1FE408FF1F00100040740BFF1F6A
:102C30003C10004000000020DC050000A022054BF5
:102C400092009B5810B5002B01D0984710BD01F0A1
:102C500003F8FBE70000FF1FA122054B92009B58E1
:102C600010B5002B01D0984710BD00F0F5FFFBE731
:102C70000000FF1FA222054B92009B5810B5002BAD
:102C800001D0984710BD00F0E7FFFBE70000FF1FF1
:102C9000A322054B92009B5810B5002B01D09847FA
:102CA00010BD00F0D9FFFBE70000FF1FA422054B79
:102CB00092009B5810B5002B01D0984710BD00F032
:102CC000CBFFFBE70000FF1F70B500F0BDFF4F4BCF
:102CD000186001F049F90400C30702D401F0A4F818
:102CE00070BD00224A4B1A604A4B187801380428FC
:102CF00029D800F013FF0320181C2400200001F045
:102D00001BF80128ECD0444C2378042B6ED101F041
:102D100093F90028E4D001F03FF9582001F00CF9B4
:102D200002232370DCE7200001F03EF8E9E72000F1
:102D300001F00AF8E5E7200001F03EF8E1E72000A5
:102D400001F03AF9DDE701F0C7F80500012808D1E4
:102D5000324B1B78053B012B03D82000FFF76EFF99
:102D6000D1E72D4B1B78022B01D0052B20D1022D52
:102D700028D12B4B9B7BAB431CD12000FFF76CFF72
:102D8000264B18780128BED16405BCD424492522DD
:102D90004B7B034205D1233A13405A425341263319
:102DA0001A000B7D9342AED9322000F0A5FFAAE7AE
:102DB000022D07D1194B1B78052B11D12000FFF7ED
:102DC00059FFDDE7012D0BD1012B03D12000FFF7C7
:102DD0005FFF98E7062B03D12000FFF767FF92E71C
:102DE000200000F039FF022D8DD1C9E7032B04D15B
:102DF0000C4B987C00F078FF72E7072B00D06FE750
:102E0000094B987B01F0D0F86AE7C0469C09FF1F88
:102E10009809FF1F9009FF1F2309FF1F1C09FF1FAF
:102E2000A60BFF1FBC0BFF1FD40BFF1FFA210A4B81
:102E30000A4A49001A640A4A5A500A4A04395A503E
:102E4000094A08319A64094A5A50094A5C315A5071
:102E5000084ADA667047C0460000FF1FF927FF1FC7
:102E6000F528FF1FA928FF1FD923FF1F6927FF1F70
:102E7000791EFF1F4D1EFF1FF7B50B0CFF27012208
:102E8000009300233C001E001D009446019089B26F
:102E900062469A401000084018413618B6B2FF2F1B
:102EA00002D1012E00D19FB2009802401A41AD1804
:102EB000ADB2FF2C02D1012D00D19CB20133102BF9
:102EC000E6D10320012E07D1012D04D1019B24015D
:102ED000E4191C700138FEBD102EFCD10238102DF3
:102EE000F9D00230F7E700008023F7B59C46264B67
:102EF000264F01932649274A274D284C284B022864
:102F00001AD1604638600868264E30408026360365
:102F10003043086001990978002909D11660224AD6
:102F20002A60224A2260E02219689143A03A1BE0FD
:102F30008021C9021160F2E766463E600F68194EB3
:102F40003E408027FF023E430E6001990978002928
:102F50000DD1176001280ED1154A2A60154A22604A
:102F6000E02219689143C03A0A431A60F7BD8021F4
:102F700089021160EEE7E0210F4A02432A600F4AFE
:102F800022601A688A43F0E74B0AFF1FE000034003
:102F9000D80003409000034000000340500003406D
:102FA00040000340FFFFE3FF0280063D804508220A
:102FB0000180063D80660822008006988055082220
:102FC000F8B51E4B80261A680020140034403242A7
:102FD00032D11A681A4F32431A6001223B68063018
:102FE00093433B6000F010FE0122164D2B681E43F8
:102FF0002E603B680A2613433B608027BF00124BBC
:103000001B683B4211D1013EF6B2FF2E09D17E2250
:103010000E4B1C682B68E40B1440934323432B6036
:1030200005E0082000F0F0FDE9E7002EEFD1802256
:103030002B68600893432B60F8BDC046C4F0004085
:103040005CF0004018F0004068F0004060F0004084
:1030500010B500F0C9FE01215820034A00F024FFFA
:10306000FFF7AEFF10BDC046600AFF1F10B5782203
:103070000021034800F058FF00F09EFD002010BD25
:103080003867FF1F70B5040000F066FD00230C20B8
:103090000B4A010059438D18515C00290DD0A14203
:1030A00008D1012300246B7000F0DEFE00F064FE06
:1030B000200070BD01330A2BEBD11224F6E7C04685
:1030C0003867FF1F70B5040000F046FD00231900AB
:1030D0001D000D4A1078002806D0A0420CD1557072
:1030E00001310C320A29F5D1002B0AD100F064FD20
:1030F00000F042FE002070BD5078461EB0411B1803
:10310000EEE700F0B1FEF3E73867FF1FF7B5040004
:103110000C20002384460E4D019267465F43E85D14
:103120007E19A04212D000280BD10A4B9C46624661
:103130001B7808331370019B70707C557160B3600D
:10314000FEBD01330A2BE8D10320F9E70720F7E79A
:103150003867FF1F3467FF1F8020F8B5484BC00554
:103160001B68C1248360474BFF251A680123134362
:103170004361454BA4001A68444B40211A60444BFC
:103180001A68444B1A60444B1A59AA431A51C52273
:1031900092009E58AE433143802699509F583F4934
:1031A000F6010F403E439E509E5880273602360A55
:1031B0003043985080201A5900020A4002431A51A5
:1031C00004341A59364E3F04324080263A431A518D
:1031D0001A5936061202120A32431A5108341A5981
:1031E00080260A4002431A51C32292009F58B446D7
:1031F000AF4337439F509F58294E0F4007439F507E
:103200009F58374080263604374380269F509F586A
:1032100036063F023F0A37439F50C0221F59AF4333
:103220003A431A511A591202120A1643C6221E5163
:1032300092009C58AC4365462C439C509C580025FA
:103240000C4020439850C72080001A58154C11405C
:10325000C02212020A431A50134B1B78DB08AB4200
:1032600001DC0020F8BD2378002B06D0A368002BDA
:1032700000D0984701350C34EEE71220F2E7C04643
:103280004C43FF1F4843FF1FB0F000403067FF1F53
:10329000B4F000402C67FF1F00E100E0FF00FFFFDB
:1032A000FFFF00FF3867FF1F3467FF1F030010B5E3
:1032B0001F2809D8072200201340072404490A7850
:1032C000A24313430B7010BD00230620F5E7C04650
:1032D0003467FF1F054B06491B780A6805485B07E2
:1032E00002401B0B134300200B6070473467FF1F25
:1032F0001CF00040FFFFC1FF70B50C25FFF7EAFF8F
:103300000A4B1C780A4BE4086543ED18002C01D1E8
:10331000200070BD2B78002B06D06B68002B00D0EE
:103320009847013C0C3DF1E71220F2E73467FF1F9C
:103330002C67FF1F1FB5002102220B000191009195
:10334000052000F099FC02230B490A681A42FCD1BF
:1033500020230393039B5A1E0392002BFAD1074AA2
:103360001368002BFCDA0B246C442000012100F0D0
:10337000C3FD207804B010BD90C8004000C80040D4
:1033800013B504000A4B0193019B002B01D11120BE
:1033900016BDFFF7CFFF23000340044205D00520F0
:1033A00000F032FC019B013BEDE71800F0E7C0465E
:1033B000FFFFFF0707B500F0CFFB80220821D205F1
:1033C000936A0191002B01D10739916202210C4AC5
:1033D00011600199481E01900029FAD10331116052
:1033E000053101910199481E01900029FAD111601F
:1033F000002B02D18022D205936200F0BDFC07BDF4
:1034000000C00040F0B52D4C89B02378002B4FD17F
:10341000FEF7D2FA02232A4F03903A681A42FCD1EF
:1034200020230693069B5A1E0692002BFAD1254EA6
:103430003368002BFCDA0120FFF7A2FF011E02D047
:10344000112009B0F0BD030003220190009005ADEA
:103450009F2000F011FC0321280000F04DFD022305
:103460003A681A42FCD120230793079B5A1E079201
:10347000002BFAD13368002BFCDA0120FFF780FF24
:103480000028DDD10398FEF7ABFAAA786B78110417
:103490001B020B4329780B4363601300113B0A495D
:1034A000052B07D801239340A3600B6001232370F1
:1034B0000020C6E780231B03F6E7C0463443FF1F06
:1034C00090C8004000C800409808FF1F1E4B30B550
:1034D0005A6818781D4B85B0D31859424B410121C9
:1034E0000093002300F0D8FB194B1A4A02259A6377
:1034F00000221A6510325A658022C4219D65164B40
:103500001648D202DA6789004258154B80241A40C7
:1035100080231B0413434350642341200393E40599
:1035200000F006FA402000F003FA6562039D6B1E6E
:103530000393002DFAD103236362FFF73BFFA562DB
:10354000FFF760FF05B030BD4043FF1F95FFFEF75A
:1035500000C80040050001FF04E100E000E100E0D8
:10356000FFFF00FFF0B585B00700FEF725FA022344
:1035700005002D4C22681A42FCD120230093009BA9
:103580005A1E0092002BFAD1284E3368002BFCDA29
:103590000120FFF7F5FE002803D01124200005B01C
:1035A000F0BD234B2360022322681A42FCD1202362
:1035B0000193019B5A1E0192002BFAD13368002B14
:1035C000FCDA0120FFF7DCFE0028E6D1194B1F6072
:1035D000022322681A42FCD120230293029B5A1E26
:1035E0000292002BFAD13368002BFCDA0120FFF79E
:1035F000C7FE0028D1D1104B2360022322681A4253
:10360000FCD120230393039B5A1E0392002BFAD173
:103610003368002BFCDA0120FFF7B2FE041EBCD198
:103620002800FEF7DDF9B9E790C8004000C8004067
:1036300001000006A8C800400180000110B500206C
:10364000FFF790FF10BD000010B5064B18705960D1
:10365000FFF73CFF00211320034AFFF757FD00202E
:1036600010BDC0464043FF1FCD34FF1FF0B504001E
:1036700085B003920291FEF79FF9882263035B0BEA
:1036800052051A438023DB059D6A8023274F009251
:10369000BA68002601901B039A420CD9F823260031
:1036A0001B041E401C4206D08022214B52025E6247
:1036B00019680A431A60002D0BD100F04DFA02225E
:1036C0001C4B1A608023DB055A62013A9A6200F0B3
:1036D00053FB0023039A934220D1002D0AD100F01E
:1036E0003BFA144B03221D608023DB055A629D6266
:1036F00000F042FB8023BA681B039A4208D9002ECF
:1037000006D000220A4B0C495A621A680A401A6015
:103710000198FEF765F9002005B0F0BD009A029906
:10372000D2181278CA540133D4E7C0463443FF1F7D
:1037300000C8004000C00040FFFFFEFFF0B587B0AA
:10374000029103920400FEF737F9019000F004FAA9
:10375000802302250122234EDB0535605D629A62DB
:1037600000F00AFB204F3B682B42FCD1202304933E
:10377000049B5A1E0492002BFAD11C4D2B68002B7F
:10378000FCDA0120FFF7FCFD002802D0112007B071
:10379000F0BD2000039A029900F0F6F9022304001C
:1037A0003A681A42FCD120230593059B5A1E0592C4
:1037B000002BFAD12B68002BFCDA0120FFF7E0FD8B
:1037C000051EE3D100F0C8F980230322DB05356034
:1037D0005A629D6200F0D0FA0198FEF701F9E0B25A
:1037E000D5E7C04600C0004090C8004000C8004077
:1037F000F0B5802489B00600FEF7DEF8E405A36A80
:1038000002250393029000F0A7F90123304F3D6099
:103810006562A36200F0B0FA2E4C23682B42FCD103
:1038200020230593059B5A1E0592002BFAD12A4DA1
:103830002B68002BFCDA0120FFF7A2FD002803D043
:103840001124200009B0F0BD244B2360022322681C
:103850001A42FCD120230693069B5A1E0692002B87
:10386000FAD12B68002BFCDA0120FFF789FD021E3C
:10387000E6D11B4B03211E60030001900090202025
:1038800000F0FAF9022322681A42FCD120230793A0
:10389000079B5A1E0792002BFAD12B68002BFCDAEB
:1038A0000320FFF76DFD041ECAD100F055F98023F7
:1038B0000322DB053C605A629C6200F05DFA039BC8
:1038C000002B01D1FFF776FD0298FEF789F8B8E7E3
:1038D00000C0004090C8004000C800400100000641
:1038E00094C8004007B5000201910422000A01A912
:1038F000FFF724FF0EBD000073B5050005240B4A39
:10390000A3005B429B1819686B46DE1D3000FFF771
:10391000B3FA022804D133782B55013CEFD276BD9F
:10392000052CFCD00128FAD10230F8E71409001167
:103930001F2807D8012380228340D20591680B43BA
:10394000936070473F2808D80123802220388340A5
:10395000D20551690B435361F3E75F28F1D8012386
:10396000802240388340D205116A0B431362E8E796
:103970001F2807D8012280218240C9058B68934304
:103980008B6070473F2808D8012280212038824070
:10399000C9054B6993434B61F3E75F28F1D80122D6
:1039A000802140388240C9050B6A93430B62E8E7E7
:1039B0001F2810D880230200DB05153A1968012A58
:1039C00006D820229143196019680A431A6070478B
:1039D00001228240F6E73F2811D880230200DB0550
:1039E000353AD968032A06D810229143D960D9689C
:1039F0000A43DA60EBE7012220388240F5E75F28CE
:103A0000E5D842238022181A413B8340D205516AEF
:103A100099435162516A0B435362D8E710B50400D1
:103A2000012813D1A022184992050B685B015B099C
:103A300013430B60154B164A19681140154A0A4387
:103A40001A60402219680A431A6010BD0028FCD190
:103A500001000A2000F060F921000B2000F05CF961
:103A6000C0220A4B920019680A4340211A601A6862
:103A70008A431A60B022044912060B685B015B0995
:103A800013430B60E1E7C04614F000401CF0004017
:103A90007F00FEFF80FD010072B6074A1368013304
:103AA00013600422054B1A600023054A136080222C
:103AB000D2055360FEE7C0467808FF1FC0F0004003
:103AC000C4F0004005490B68002B05D1044A0A6088
:103AD00004490A60044A13607047C046140AFF1F75
:103AE000841E0000380AFF1FC4F000400023034A70
:103AF0001360034A1360034A1360704754F0004098
:103B000040F1004044F1004002B4714649084900C8
:103B1000095649008E4402BC7047C04602B4714643
:103B200049084900095C49008E4402BC7047C04600
:103B300003B47146490840004900095A49008E44BF
:103B400003BC70470000000001B40248844601BC79
:103B5000604700BF8D11010001B40248844601BCDA
:103B6000604700BF75A9000001B40248844601BC4B
:103B7000604700BFED6B010001B40248844601BC00
:103B8000604700BFE927000001B40248844601BC39
:103B9000604700BF9573010001B40248844601BC30
:103BA000604700BF2D6C010001B40248844601BC8F
:103BB000604700BFC166010001B40248844601BCF1
:103BC000604700BFADAE000001B40248844601BCAE
:103BD000604700BFEDA5000001B40248844601BC67
:103BE000604700BF8914010001B40248844601BC4B
:103BF000604700BFCD4C010001B40248844601BCBF
:103C0000604700BF090E000001B40248844601BCB1
:103C1000604700BF0189000001B40248844601BC2E
:103C2000604700BFE512010001B40248844601BCB0
:103C3000604700BFDD3F000001B40248844601BC7C
:103C4000604700BF8552010001B40248844601BCB0
:103C5000604700BFC95C010001B40248844601BC52
:103C6000604700BFE917010001B40248844601BC67
:103C7000604700BF8512010001B40248844601BCC0
:103C8000604700BF496D010001B40248844601BC91
:103C9000604700BF2144000001B40248844601BCD3
:103CA000604700BFC56D010001B40248844601BCF5
:103CB000604700BF9D6A000001B40248844601BC11
:103CC000604700BF7997000001B40248844601BCF8
:103CD000604700BFC115010001B40248844601BC21
:103CE000604700BF6911010001B40248844601BC6D
:103CF000604700BF4DF9000001B40248844601BC92
:103D0000604700BF6137010001B40248844601BC2E
:103D1000604700BF8937010001B40248844601BCF6
:103D2000604700BF85A3001101B40248844601BC6E
:103D3000604700BFD544010001B40248844601BC7D
:103D4000604700BF0134010001B40248844601BC51
:103D5000604700BF0534010001B40248844601BC3D
:103D6000604700BF8D82000001B40248844601BC58
:103D7000604700BF5976010001B40248844601BC87
:103D8000604700BF9DA9000001B40248844601BC01
:103D9000604700BFC9A9000001B40248844601BCC5
:103DA000604700BFE9F6000001B40248844601BC48
:103DB000604700BF0934010001B40248844601BCD9
:103DC000604700BFF535010001B40248844601BCDC
:103DD000604700BF6D0B010001B40248844601BC7E
:103DE000604700BFB352010001B40248844601BCE1
:103DF000604700BFED68010001B40248844601BC81
:103E0000604700BF156B010001B40248844601BC45
:103E1000604700BFD9B0000001B40248844601BC2D
:103E2000604700BFCD0C010001B40248844601BCCC
:103E3000604700BFDD0A010001B40248844601BCAE
:103E4000604700BF8944000001B40248844601BCB9
:103E5000604700BF090E000001B40248844601BC5F
:103E6000604700BFE94C010001B40248844601BC30
:103E7000604700BF21A9000001B40248844601BC8C
:103E8000604700BFBD5C010001B40248844601BC2C
:103E9000604700BF016C010001B40248844601BCC8
:103EA000604700BF116E000001B40248844601BCA7
:103EB000604700BF0167010001B40248844601BCAD
:103EC000604700BF75F8000001B40248844601BC99
:103ED000604700BFE9D4000001B40248844601BC39
:103EE000604700BFDD0C010001B40248844601BCFC
:103EF000604700BF85C1000001B40248844601BC90
:103F0000604700BF3D71010001B40248844601BC16
:103F1000604700BF53B9000001B40248844601BCA9
:103F2000604700BFF90D010001B40248844601BC9E
:103F3000604700BFB70E000001B40248844601BCD0
:103F4000604700BF7912010001B40248844601BCF9
:103F5000604700BFA9D8000001B40248844601BCF4
:103F6000604700BF19FA000001B40248844601BC52
:103F7000604700BFBD0B010001B40248844601BC8C
:103F8000604700BFC1A5000001B40248844601BCDF
:103F9000604700BFD1AE000001B40248844601BCB6
:103FA000604700BF6DF6000001B40248844601BCC2
:103FB000604700BFC1F7000001B40248844601BC5D
:103FC000604700BFF935010001B40248844601BCD6
:103FD000604700BF71B0000001B40248844601BCD4
:103FE000604700BF2DB7001101B40248844601BCF0
:103FF000604700BF0D52010001B40248844601BC75
:10400000604700BFF9ED000001B40248844601BCDE
:10401000604700BFE90B010001B40248844601BCBF
:10402000604700BF8B52010001B40248844601BCC6
:10403000604700BF51B8000001B40248844601BC8B
:08404000604700BF01D700003A
:1040480002000000EEBF001101000000E0BD0011F9
:1040580002000000EABF0011010000008840FF1FB5
:1040680002000000E8BD001101000000C861FF1F48
:1040780002000000E8BF0011030000003C61FF1FC0
:104088001200000002000000EEBF00110100000055
:1040980028BE001102000000EABF00110100000064
:1040A80025BE00110200000032BE0011030000000E
:1040B8007761FF1F02000000E8BF00110300000045
:1040C8008C61FF1F02000000EABF00110100000020
:1040D80024BE00110200000030BE001103000000E1
:1040E8004D61FF1F02000000E8BF0011030000003F
:1040F8006E61FF1F02000000EEBF0011010000000A
:104108006CBE001102000000EABF001101000000AF
:10411800D141FF1F020000007EBE00110100000017
:1041280063BE001102000000EABF00110100000098
:10413800D041FF1F020000007CBE001101000000FA
:104148009461FF1F02000000EABF00110100000097
:10415800CF41FF1F020000007ABE001101000000DD
:1041680053BE001102000000EABF00110100000068
:10417800CE41FF1F0200000078BE001101000000C0
:104188004EBE001102000000EABF0011010000004D
:10419800CD41FF1F0200000076BE001101000000A3
:1041A80049BE001102000000EABF00110100000032
:1041B800CC41FF1F0200000074BE00110100000086
:1041C80044BE0011020202020202000000000000C8
:1041D800161500009D4C0011634C0011DCBE001147
:1041E80090011D0018001800FFFF070102030405D5
:1041F80006020106000000000000000000000000A8
:1042080000000000000000000000000000000000A6
:104218000300000002000000EEBF001101000000D2
:10422800FCBE001102000000EABF001101000000FE
:104238008C42FF1F0200000006BF001101000000B1
:10424800C261FF1F02000000E8BF00110300000068
:104258002C64FF1F02000000EABF001101000000EB
:104268008C42FF1F0200000004BF00110100000083
:10427800C461FF1F02000000E8BF00110300000036
:104288002464FF1F120800000000000000C6C600DA
:1042980000000000000000001311000000010000F1
:1042A80000000111FFFF00005048593600000000CF
:1042B800000000000B000500F0000000B40000281A
:1042C800002800283075A000A000A000A000000869
:1042D8000008E001F00010001000100010001000AD
:1042E800100050005000500010001000D0070000CF
:1042F800000000000F0001000500307507001000E5
:10430800010081FF00000000FF0000006D75001132
:104318007573001105710011FFFF0100FF00000017
:10432800899F0011059D00111D9C001100000000CF
:104338000000000000000800040000003B00010825
:104348005902E00188212800FF0000000200000057
:10435800EEBF001101000000B4C00011020000000F
:10436800EABF001101000000D143FF1F0200000056
:10437800E6BF001101000000F067FF1F0200000007
:10438800EABF001101000000D043FF1F0200000037
:10439800E4BF001101000000CE43FF1F020000002F
:1043A800EABF001101000000CC43FF1F020000001B
:1043B800E2BF001101000000C443FF1F18001800ED
:1043C8001D0090010200000302020000020000002C
:1043D800EEBF001101000000C8C00011020000007B
:1043E800EABF0011010000001444FF1F0200000092
:1043F800E0BF001100000000000000000200000003
:0E440800E8BF0011030000001068FF1F20FF36
:040000051FFF184180
:00000001FF
